:1090E500414952434F54454300405621332E3131B7
:1090F50020454E470042415454004241440040320D
:1091050044400040334440004F4646214E455740B9
:109115004D454E55000A16000180000300007E00F3
:1091250000FE00001E0000360003E60001C400003A
:1091350000000FFFE053454152434840534154530B
:109145000043414C40414C544920202300504943A1
:10915500545552450052414E4B494E47004D4150E2
:109165002020200043454E54455200564152494F58
:1091750020004241524F475200524F55544553002B
:109185004E454152535400574159505453004D4197
:10919500524B53200044454641554C540020202055
:1091A5002141564721202020204453540021455871
:1091B50049540153454C40524F555445015345546C
:1091C5002048454947485401464C4947485453208F
:1091D5006869015741595054532020686901524F1D
:1091E5005554455320206869014149525350414324
:1091F5004568690153455454494E475368690053BE
:10920500455420484549474854004241524F40483B
:109215004549474854004750532048454947485415
:1092250000514E4820202020402148504100464C06
:10923500004C4F47424F4F4B20454D505459003E2F
:109245002145584954002145584954015245504C2F
:1092550041590153454E440144454C45544500216F
:109265004558495401544E432031232035374B018D
:10927500544E4320312320392E36010150574340A7
:109285003130234035374B0150574340313023406F
:1092950031394B01014D5850403130234035374B62
:1092A500014D58502034232035374B014D5850205F
:1092B50031232035374B014D585040313023403153
:1092C500394B014D58502034232031394B014D582D
:1092D500502031232031394B002145584954014E46
:1092E500455720205741595054014544495420576A
:1092F500415950540144454C20205741595054017F
:1093050001434F4D3A015245434549564520575073
:109315000153454E442057415950540153454E443D
:1093250040414C4C4057500101444953542057503B
:109335002D57500144454C40414C4C40575054002A
:109345004252472021444953540053544F5245003B
:1093550050524553454E5440504F532E005550449E
:109365004154494E472E2E004044454C45544544F2
:1093750000534552200049524441005553422000B4
:1093850020425420004C4953540053454E4400207C
:109395005452414E534D4954204552524F5220008C
:1093A50021455849540153454C40524F55544501A8
:1093B5004E455720205254455054014544495420A8
:1093C500524F555445015245564552534520525426
:1093D5000144454C202052544550540144454C20ED
:1093E50020524F5554450101434F4D3A01524543D3
:1093F500454956452052540153454E4420524F5538
:1094050054450053454C21524F555445004E404557
:10941500405700204E455740504F534021002140B2
:109425005245564552534540005245565253002128
:109435004044454C405750545300214044454C202E
:10944500525445004E4F5420454D5054592000214B
:0D9455004053454E444052544500214558B7
:109462004954014C4F414440435452215043015608
:10947200494557404354520144454C40414C4C21CC
:109482004354520101434F4D3A0152454356202065
:109492004354520153454E442020435452005649EE
:1094A2004557204354520020204D4F56450020205E
:1094B2004D4F564520544F005343414C45202058B0
:1094C2002F5920204558495400434C5220444953B7
:1094D20054004155544F43454E54004155544F207A
:1094E2004F4646002020205343414C4500444953F7
:1094F20054204B4D0044495354204E4D00214558B1
:10950200495401564152494F20202068690158436D
:109512002D53455420206869015254452D5345541A
:109522002068690147454E4552414C206869015007
:109532004943545552455368690101014541535904
:109542002D53455401464143544F525921534554DA
:109552000144454D4F464C494748540144454C212E
:10956200414C4C21464C490021455849540153492C
:109572004E4B544F4E450153494E4B212D015349F9
:109582004E4B404D4F440153494E4B40494E5601BC
:10959200564152205443402020402301564F4C55FF
:1095A2004D4501564152494F204E554C4C015049B0
:1095B20054434801504552494F44015641522041BB
:1095C2005640203040230154454320202040303073
:1095D200402501534F554E44434845434B005349A0
:1095E2004E4B21544F4E450053494E4B54214F464A
:1095F20046004E4F542150524553454E5400564159
:1096020052494F204E554C4C004B45455040515508
:10961200494554403130404D494E004245464F5233
:1096220045204E554C4C494E47002145584954015E
:109632004D415021545241434B014155544F4345F2
:109642004E5401014156472F4449535401474C445B
:109652004550415448014C2F44010157494E442181
:10966200542D55500143454E5421542D555000213F
:10967200455849540153544152544054494D4501AF
:1096820046495253540144454C544120203A014D1D
:10969200554C5449504C45014C41535401015345DA
:1096A2004C40524F5554450101010143594C52015E
:1096B20043594C20542D555000214558495401011D
:1096C200554E495401434C49434B40302C402023D2
:1096D20001434F4E5452415354014E4D45412131A5
:1096E200383301494D50454C4C4552004057415981
:1096F200504F494E54204558495354534000574106
:1097020059504F494E540020204558495420202199
:109712000052454345495645004652454540004E94
:1097220045585420545054005052455620545054D9
:1097320000434C5220404C454700434C522040537A
:10974200554D004F4646202020202020202000207A
:109752004F464600475053204552524F52005354F1
:109762004F52494E4700524F555445004E454152C3
:10977200455354004C495354200045544500414C34
:1097820054403000454D5054592052544520002039
:10979200544F4F404D5543482000214053454C40C3
:1097A2004C495354002053454C40575054402100DB
:1097B20021405245434549564540002020404F2014
:1097C2004B40202021004F4B0020204641494C2095
:0D97D20020210020455849540045444954C9
:1097DF00005940454053004544495420204E4557B9
:1097EF00202053544F5245004E4558542053454C5A
:1097FF004543542045584954005843542D464C492D
:10980F0047485420005553454400454E5445522077
:10981F00004D4D2E4D4D4D20004D4D2753532E5382
:10982F0000574753213834002040554054404D4095
:10983F002000554054404D002055544320004C4FBC
:10984F0043414C005357495353474400414C540034
:10985F00535549405800415647402030402300356A
:10986F003030003136343000205D203130404B63D2
:10987F002F70005D2020203140632F2300205D20BA
:10988F002035404B5453005D203230304046504D10
:10989F0000406340204B63004654204B63004063FD
:1098AF0040204E4D004654204E4D004D2F53003258
:1098BF0030305E003530305E00312200322200330E
:1098CF002200352200382200464C3700464C3136F4
:1098DF0000464C333300464C3635004631303000AD
:1098EF00463136300046323630005E252640534F23
:1098FF0047005E25264054415300414C54005641C9
:10990F005200225E2F24004B545300532F4E00223F
:10991F0024004B5400225E004E4D00302C35003198
:10992F002C3000322C3000302C3600312C320032EB
:10993F002C3500332C3800372C35004031350040A2
:10994F003330004036300020545241434B214F4EAC
:10995F0020200020545241434B214F464620003CCB
:10996F002D204C495354202D3E202045584954005A
:10997F0053454C004E455854005441534B00464CF0
:10998F002D4441544500545000544F460053544108
:10999F000046494E004C414E00534554204F464619
:1099AF005345540049534120484549474854004DB9
:1099BF0041524B0020545241434B2D555021200012
:1099CF00204E4F5254482D555021200056415200E1
:1099DF004649580047415445215800535441525469
:1099EF004C494E452000535443594C2000404F469C
:1099FF00460054502000406A40494E2000406740C6
:049A0F004F5554005B
:10497900304D2475A7049005C2E0F51CE0F51DE053
:10498900F51EE0F51FE0F56DE0F56EE0F56FE0F579
:104999005412553B124F792275C70375C6E475B990
:1049A90001E5BCB4814312553B125F458E628F63AA
:1049B9007568F9756900124A4F203C2D203B2B126E
:1049C9004B84124B58856D1C856E1D856F1E855451
:1049D9001F124ABB203C12203243201D23124B8454
:1049E900124F79E532242850DC22124ABB203CF9C7
:1049F900203DF6203205201DBD80EF301DB880EA2C
:104A0900124B84124F79856D1C856E1D856F1E852D
:104A1900541F124B6E124F79203DCE8099124DA72B
:104A2900201D0D7553107400124D0A203DBB808660
:104A3900E553540FC553C4540F203505124C1F803C
:104A490003124D0A808BC23CD23B124B0BFD124B19
:104A59000BFC124B0BC39573F565EC9574F564ED7E
:104A69009575600504600A800EE56424E0501180A4
:104A790006E56424204009124B0B124B0B024B0B29
:104A8900124B0BFD124B0BFC124B0BC39576F567C2
:104A9900EC9577F566ED9578600904600122E56685
:104AA900F48002E5668562F0A474E025F04002C254
:0D4AB9003B22C23C124B0BA2E7923DA2E64D
:104AC600921DA2E592324026A2E492E592E692E792
:104AD600FC124B0B2565F565EC3564F564124B0B42
:104AE600FC124B0B2567F567EC3566F56622A2E4EA
:104AF6009235540F79C6F7124B0B09F7301D051284
:104B06004B0BF55322E5697023E5686030240340BA
:104B16002CE56875F004A485F0C7F5C675B901E5FE
:104B2600BCB4811985BD68756902801E5403701076
:104B360005C675B901E5BC056953690F22D23C2249
:104B4600147004E5BD80F0147004E5BE80E9E5BF8D
:104B560080E575A7009006F6E56DF0A3E56EF0A377
:104B6600E56FF0A3E554F02275A7009006F6E0F590
:104B76006DA3E0F56EA3E0F56FA3E0F55422E564BE
:104B8600B2E7F56D85656EAB67E566FC30E707C392
:104B9600E49BFBE49CFCAA62A963125C5FE56630B9
:104BA600E707C3E49DFDE49EFEEEB2E7F56F8D5484
:104BB6002275380C124E10124E5BD55301227538F1
:104BC6000C124DE1124E51D5530122753800124D8B
:0E4BD600F9124E20D5530122753800124DE120
:104BE400124E20D5530122753803124E10124E8CEA
:104BF400D5530122753803124DE1124E82D553016B
:104C04002275380F124DF9124EB1D5530122753861
:104C14000F124DE1124EB1D5532622904C2423732A
:104C24008091807780688059804A803B802C801DE9
:104C3400800E80DA80CB80BC80AD809E808F8080A7
:104C4400753815124E10124ED3D5530122753815EE
:104C5400124DE1124EC8D5530122753809124DF98F
:104C6400124E99D5530122753809124DE1124E990D
:104C7400D5530122753806124E10124E43D55301F6
:104C840022753806124DE1124E38D553012275387B
:104C940012124DF9124E69D5530122753812124D74
:104CA400E1124E69D5530122024BB7753815124EE5
:104CB40010124ED3D553012275380F124DE1124E06
:104CC400B1D553012275380F124DF9124EB1D55397
:104CD4000122753803124DE1124E82D5530122751B
:104CE4003803124E10124E8CD5530122753800121F
:104CF4004DE1124E20D5530122753800124DF912A0
:104D04004E20D5532622904D0F2373809E80A98078
:104D1400B480BF80CA80D580E08010801B8026804C
:104D240031803C80478052805D806875380C124D1C
:104D3400E1124E51D553012275380C124E10124E09
:0E4D44005BD5530122753812124DE1124E69F3
:104D5200D5530122753812124DF9124E69D55301FD
:104D620022753806124DE1124E38D553012275389C
:104D720006124E10124E43D5530122753809124DB8
:104D8200E1124E99D5530122753809124DF9124E8E
:104D920099D5530122753815124DE1124EC8D553DB
:104DA2000122024CAF78C686040886037AED125CB3
:104DB2001D78CAA60408A60378C686040886037A64
:104DC20062125C1D78CCA60408A60378C686040885
:104DD20086037AB5125C1D78C8A60408A60322755C
:104DE2001A6A751B0A78CA8618088619125024781E
:104DF200CC86060886072278C88618088619E4F544
:104E02001AF51B12502478C886060886072278C62F
:104E12008618088619751A00751B01025024E51DB3
:104E22002519F51DE51C3518F51CC3E51F9FF51F57
:104E3200E51E9EF51E22C3E51F9FF51FE51E9EF58A
:104E42001EC3E51D9519F51DE51C9518F51C22E5F7
:104E52001D2FF51DE51C3EF51CC3E51F9519F51F19
:104E6200E51E9518F51E22C3E51D9FF51DE51C9E46
:094E7200F51CC3E51F9519F51F9D
:104E7B00E51E9518F51E22E51F2FF51FE51E3EF5C5
:104E8B001EE51D2519F51DE51C3518F51C22C3E57E
:104E9B001D9519F51DE51C9518F51CE51F2FF51F24
:104EAB00E51E3EF51E22E51D2FF51DE51C3EF51CEE
:104EBB00E51F2519F51FE51E3518F51E22C3E51D47
:104ECB009FF51DE51C9EF51CE51F2519F51FE51E1D
:104EDB003518F51E22E51A7009E51B70058C068D39
:104EEB000722ED851BF0A4A2F792D5ED851AF0A44D
:104EFB00AEF0FFEC851BF0A4A2D53FEE35F0FF9290
:104F0B00D5EC851AF0A42FFFE435F030D50104FE63
:104F1B0022E4F51AF51BEF4E7003051B22EF651902
:104F2B007006EE65187001227808C3EF33FFEE337D
:104F3B00FEEF9519F5F0EE95184003FEAFF0E51A6C
:104F4B0033F51AD8E5F4F51A751BFF7805C3EF3363
:104F5B00FFEE33FEEF9519F5F0EE95184003FEAF1B
:034F6B00F0E51B53
:104F6E0033F51BD8E5F4C403F51B22E51D9511E5B9
:104F7E001C9510500BE56E9511E56D9510500122A4
:104F8E00E51F9511E51E9510500BE5549511E56F33
:104F9E009510500122E51D9513E51C9512400BE569
:104FAE006E9513E56D9512400122E51F9513E51ED2
:104FBE009512400BE5549513E56F9512400122535F
:104FCE002CF8C3E51F9554FFE51E956FFE926050B9
:104FDE0007C3E49FFFE49EFEC3E56E951DF519E53C
:104FEE006D951CF5189261500BC3E49519F519E4F3
:104FFE009518F518C3E5199FE5189E9262500AE5BB
:10500E0018CEF518E519CFF519124F1CE52C5407DB
:10501E0075F003A4F538E53890502A730250420219
:10502E00505602506402507C02508F0250A2025021
:10503E00B00250C8851C16851D17C3E4951FF515C3
:10504E00E4951EF5140250DB851C16851D17851E72
:10505E0014851F158077C3E4951DF517E4951CF58F
:10506E0016C3E4951FF515E4951EF514805FC3E491
:05507E00951DF517E48B
:10508300951CF516851E14851F15804CC3E4951FCA
:10509300F517E4951EF516851C14851D15803985B5
:1050A3001E16851F17851C14851D15802BC3E495BB
:1050B3001FF517E4951EF516C3E4951DF515E49544
:1050C3001CF5148013851E16851F17C3E4951DF563
:1050D30015E4951CF5148000C3E5179513E51695A3
:1050E3001210D70122E5159513E514951210D70177
:1050F30022E519F92517FFE518F83516FED3EF95C4
:1051030011EE9510500122E5119517FDE510951646
:10511300FC402A4D6027124EE0E5152FF515E514E6
:105123003EF514E5159513E514951210D70122E504
:10513300199DF9E5189CF8851016851117E51729AF
:10514300FFE51638FEE5139FE5129E500BC3E513EA
:105153009517F9E5129516F8E51A700AE51B70061E
:10516300AA00AB018013E9851AF0A4E5F0FBE885FA
:105173001AF0A42BFBE435F0FAE5152BFBE5143A02
:06518300FAE5119BE510A6
:105189009A10D70122EB9515FDEA9514FCC3E51594
:105199009511E514951010D717E5139BE5129A5050
:1051A90036E5139515FFE5129514FE12545880271C
:1051B900EB9511FFEA9510FEAA00C001125458D0D0
:1051C90003E5172BFBE5163AFAEB99F517EA98F57B
:1051D90016851115851014C2D5E5466002D2D5AAE7
:1051E90056E98AF0A4ABF0E88AF0A42B30D504750F
:1051F900F00384F8700122E5172513FDE516351231
:10520900FCED8AF0A4ABF0EC8AF0A42B30D5047540
:10521900F00384FEE5152513FDE5143512FCED8A2E
:10522900F0A4ABF0EC8AF0A42B30D50475F003841C
:10523900F9E5389052407302525802526402526D95
:1052490002527602527C02528802528F025294C351
:10525900743E9EFFC3743E99FE8032C3743E9EFF26
:10526900AE018029AF06C3743E99FE8020AF06AE19
:0D52790001801AC3743E9EFEC3743E99FF6F
:10528600800EC3743E99FF8007C3743E9EFEAF0135
:1052960008EF2437FFE51B7007E51A700CE8800E4F
:1052A600A2E7E51A50030460F488F0A4E5F0600173
:1052B60004F923FA98FBC3E998C333F99052C8E579
:1052C60038730252E002530D02534202536F0253E7
:1052D6009C0253C90253F602542305A7800BEB30F8
:1052E600E7032A8002291E1FFBEEC45403F583EE52
:1052F6005408C42FF582EE5407243883F5F0E045B0
:10530600F0F0D8DA05A72205A7800BEB30E7032AD1
:105316008002290E1FFBEEC45403F583EE5408C425
:105326002FF582EE5407240B83F5F0E045F0F0D814
:10533600DA05A722804020100804020105A7800B89
:10534600EB30E7032A8002291E0FFBEEC45403F557
:1053560083EE5408C42FF582EE540724EC83F5F04F
:10536600E045F0F0D8DA05A72205A7800BEB30E779
:05537600032A8002295A
:10537B000E0FFBEEC45403F583EE5408C42FF582D5
:10538B00EE540724BF83F5F0E045F0F0D8DA05A71B
:10539B002205A7800BEB30E7032A8002291F1EFB97
:1053AB00EEC45403F583EE5408C42FF582EE540774
:1053BB00249283F5F0E045F0F0D8DA05A72205A793
:1053CB00800BEB30E7032A8002291F0EFBEEC4543F
:1053DB0003F583EE5408C42FF582EE54072465833E
:1053EB00F5F0E045F0F0D8DA05A72205A7800BEB26
:1053FB0030E7032A8002290F1EFBEEC45403F5830A
:10540B00EE5408C42FF582EE5407243883F5F0E0F0
:10541B0045F0F0D8DA05A72205A7800BEB30E703A0
:10542B002A8002290F0EFBEEC45403F583EE5408B9
:10543B00C42FF582EE5407240B83F5F0E045F0F012
:10544B00D8DA05A7228040201008040201EC701F57
:08545B00ED20E740D2E023CF71
:1054630023CF30E7F980357B08801A7B1080167BC9
:105473002080127B40800E20E4ED20E3EE20E2EF5B
:1054830020E1F07B80EE8BF0A4CF8BF0A4E5F02F2E
:10549300FFEC8BF0A4CD8BF0A4E5F02D2499838F42
:1054A300F0A433E5F033FBE98BF0A4E5F0C88BF00F
:1054B300A428F9E435F0F822FFFEFCFAF8F6F4F23A
:1054C300F0EFEDEBEAE8E6E5E3E1E0DEDDDBDAD998
:1054D300D7D6D4D3D2D0CFCECCCBCAC9C7C6C5C4F6
:1054E300C3C1C0BFBEBDBCBBBAB9B8B7B6B5B4B310
:1054F300B2B1B0AFAEADACABAAA9A8A8A7A6A5A4FC
:10550300A3A3A2A1A09F9F9E9D9C9C9B9A999998BF
:105513009797969594949392929190908F8F8E8D66
:105523008D8C8C8B8A8A89898887878686858584F2
:10553300848383828281818075A700905561E546CB
:10554300FA24FA50027A05EA2323F978107F0493A8
:10555300F60809E9DFF9905579EA93F556227FC2F7
:10556300803E7F4680BA7E8C81747D1882E87A30D3
:1055730085D074608BA0808040201008125585026E
:1055830057DBD215D274D273C219C23A125F458E59
:1055930047757D007546057552021285C112021FBB
:1055A300E53524EB500E1285C17F199094CB126B15
:1055B300FA12D026E55275F016A4F57012579175BC
:1055C300511512565C7F237E099094A9126C0C121C
:1055D300D02610000810010D10021280E2125704A9
:1055E30075330180DA12574975330180D275510042
:1055F30012565C7E009094BA126C3F7F237E059016
:1056030094B0126C0C1256AD12D026E55210000F56
:1056130010010510028780D5045403F55280CE1281
:10562300565C7F237E0B9094E8126C0CE546600772
:1056330014600414123C3D12D026E54610000810F5
:10564300010B10021180D860D6154680D2B4050232
:1056530080CD054680C90255A075320012D1E67F80
:10566300017E119094A0126C3F7E0012C840E55158
:10567300D26612C89775170812CCCE123C75757195
:1056830000C20612C9E7741BFFF5177E0F9094EF53
:10569300305D039094F7126C3F1286041265011279
:1056A300419EC2061249A102189FE552601414607C
:1056B3001E1460297F647E2D791C1256F71E1FD994
:1056C300F9227F6A7E1F79281256F71FD9FA227FA3
:1056D300487E2D791C1256F70F1ED9F9227F567E6C
:1056E3003379281F12D12B0F0F12D12B1F12D12B5D
:1056F3001ED9F0221E12D12B0E0E12D12B1E02D157
:105703002BE552605514606814606D800075709EBF
:1057130012577E8003757000E5732540F573E435F9
:1057230074F574E43575F5752275701612571B8080
:105733000375702DE5762542F576E5773541F577E6
:10574300E43578F57822E55260CB1460DC1460E12F
:105753008000757044125737800375705AE573954E
:0957630040F573E5749400F5743F
:10576C00E5759400F575227570711257608003759C
:10577C007088E5769542F576E5779541F577E5788D
:10578C009400F57822E5469057A793F540FEAD4777
:10579C00E4FFFC125CF28E418F4222020C18306046
:1057AC00C07F401209A51218B512D026125A51EB1F
:1057BC00700590923D800B1258649097BD500390E9
:1057CC0097CB7F3F7E04126C0C12D02612D0B212F3
:1057DC00D0E275370990945F1217A09057EB7302C3
:1057EC0002970259AB02557F025A820257DB0258CC
:1057FC000302581C0257AD7F2E12113580D17F3613
:10580C007E04909791126C0C12D02612D0B280BFED
:10581C007F371209A51218B512D026125A35124329
:10582C001ED2AC1000A9306DFA125914203BCF4097
:10583C00ED7568F975160012596140FB125AFD7F1F
:10584C00367E29E51612C61E12D0260516126CB22B
:10585C0078C6B6F7E2025A2F7C0512431E12CDD041
:10586C00744112CE03745312CD9EEB12CDBF126C49
:10587C00C45003DCE5227515F975160010000EE511
:10588C001560251258B640051258DD5002D3227F00
:10589C003F7E29E51612C61E12D0267F1412D0C9DF
:1058AC000516E51664F870D4C32212723575B90169
:1058BC00E5BCB4811AE5BDF51570037516F778C60D
:0B58CC00A61612737E1273761273761C
:1058D700C3027376D3227F0575F019D5E0FDD5F0A5
:1058E700FA12431E12CDD0744112CE03744212CD68
:1058F7009E7E0F78C6E60812CD9EDEF912CDC21243
:105907006CC4400122DF012275F00080CEC23B1239
:10591700431ED2AC12CF30204C3CB440F712CF35E7
:10592700B4400312CF35B4412DF53812CF35B453F7
:105937002512CF35FA12CF35E538701A12CF35B4A4
:105947000D1412CF35B40A0EC3E5169A4003026C44
:10595700A9C2ACD23B22C2ACD322126D0812431E9D
:10596700D2AC1000F112CF30204CEBB440F412CF80
:1059770035B4400312CF35B441DCF53812CF35B416
:1059870042D47E1078C612CF35F608DEF9E53870B6
:10599700C512CF35B40DBF12CF35B40AB9C2ACC3E7
:1059A700220257DB7F0A1209A51218B512D0261258
:1059B7005A35124370D2AC1000E712CF35B440F518
:1059C700F53812CF35B46EED12CF35E538600A12CF
:1059D7004370744F12CDAA80DC12CDFEE51612CDAE
:1059E700AA12CDB47568F9751600124370D2AC10BF
:1059F700003912CF35B440F7F53812CF35B44EC55C
:105A07007E1078C612CF35F608DEF9124370E538F6
:105A17006007744F12CDAA80D1125AFD0516745132
:105A270012CDAA78C6B6F7C2125A9E0257DB751571
:0C5A37000075160412722C75B901E5BC54
:105A430030E70205160515E515242050EB227B00EF
:105A53007515F912723575B901E5BCB481010B05F1
:105A630015E515240350EC75150112722C75B90157
:105A7300E5BCB481010B0515E515242050EC227F0C
:105A83001C1209A51218F812D02610000B100102DF
:105A930080F87515F9125A9E0257DBE51560372415
:105AA30003401A241E5019E51524074002802712CB
:105AB3007235125ADA0515E515240350F2751501EE
:105AC30012722C75B901E5BC30E703125ADA0515D9
:105AD300E515242050EA22125AEF1248EE05C612A9
:105AE30048EE05C61248EE05C60248EE74FF800173
:105AF300E4F5BCF5BDF5BEF5BF22E568606AF515B2
:105B03000515E5152403501D75150112722C75B981
:105B130001E5BC30E70280190515E515242050EB9B
:105B2300751500800C241D60F750E0E51524065020
:105B330037E56875F004A485F0C7F5C675BC81E543
:105B430015F5BDF56878C6B6F70375BD0008125B99
:105B530060125B5A125B5A86BC0886BD0886BE0873
:095B630086BF081248EE05C622B7
:10B4490012A23012B54812774812B4CD12775012B1
:10B45900B4DA02A23412A23012B5481277487F5AE0
:10B46900C23C12762A127826783F79437F607EEAB9
:10B4790012B53C1277507F6512762A127826783DEC
:10B4890079417F207E4E12B53C303C2012B6FE1227
:10B49900B559783F794312B4B8783D794112B4B8B7
:10B4A90012B6FE78D7E65480F67537000287D6C300
:10B4B900E796FF1819E796FE0809C3E69FF71819DA
:10B4C900E69EF7227F5B7E0690985F126C3F1F8095
:10B4D9000A7F667E14745912C7371F1274B37E39F6
:10B4E900E402C7567866E620E73418C3E694720882
:10B4F900E694045029C318E6941F08E69404401EF4
:10B509007869E620E71818C3E6940E08E694015016
:10B519000DC318E6947508E694004002D322C322AD
:10B52900E67D0030E7011D08E62BFB18E63CFCE44C
:0EB539003DFD22C3EB9FF6F71819EC9EF6F7C6
:10B547002212B4ED400CE47842F608F67840F6088B
:10B55700F6227864C3E6946AF55708E6944CF556E4
:10B567000808C3E69458F55B08E694AEF55A7539B2
:10B5770000AC56AD57EC12A5DD784C12A66BAC5A51
:10B58700AD5BEC12A5DD785012A66B7F2B7E867D16
:10B59700777C1812A5A2785012A65F12A4AE12A546
:10B5A700A2785012A65F12A4AE12A5A2785012A6D6
:10B5B7005F12A4AE12A5A27F367E847D257C64121D
:10B5C700A5A2785012A65F12A4AE12A5A2784C12BB
:10B5D700A65F12A4AE12A5A27F3F7EA27D607C8BE0
:10B5E70012A5A2785012A65F12A4AE12A29C12A2B4
:10B5F7009C12A6777F3F7E807D057CE6053912A4E5
:10B60700AE784812A66B7F2C7E937D477C7F12A570
:10B61700A2785012A65F12A4AE12A5A2785012A665
:10B627005F12A4AE12A5A2784C12A65F12A4AE12A6
:10B63700A5A27F357EB47DF87CDF12A5A2785012D3
:10B64700A65F12A4AE12A5A2785012A65F12A4AEEE
:10B6570012A5A27F3F7EED7D227CCD12A5A2784C5C
:10B6670012A65F12A4AE12A2A012A29C784412A640
:10B677006B7F317E397D9D7CE712A5A2784C12A69F
:10B687005F12A4AE12A5A2784C12A65F12A4AE1246
:04B69700A5A27844AC
:10B69B0012A65F12A2A012A5A27F2C7E377D0C7C76
:10B6AB00A312A5A2784C12A65F12A4AE12A5A27883
:10B6BB004C12A65F12A4AE12A5A2784C12A65F1272
:10B6CB00A4AE12A2A012A6777F3F7E807D027C9F44
:10B6DB00053912A4AE784412A66B784812A65F12F5
:10B6EB00A6148E428F43784412A65F12A6148E4086
:10B6FB008F4122753900AC42AD43EC12A5DD784881
:10B70B0012A66BAC40AD41EC12A5DD784412A66BD2
:10B71B007F2B7E537D507C0912A5A2784812A65F21
:10B72B0012A4AE12A5A2784812A65F12A4AE12A55F
:10B73B00A2784412A65F12A4AE12A5A27F347EF2A9
:10B74B007DCD7CA312A5A2784812A65F12A4AE12DF
:10B75B00A5A2784812A65F12A4AE12A5A27F3F7EC7
:10B76B000A7D2E7CAE12A5A2784412A65F12A4AE5F
:10B77B0012A29C12A29C784C12A66B7F2B7E4F7D43
:10B78B00AF7CB212A5A2784812A65F12A4AE12A586
:10B79B00A2784812A65F12A4AE12A5A2784812A6F0
:10B7AB005F12A4AE12A5A27F357EB17D4B7C9512A4
:10B7BB00A5A2784812A65F12A4AE12A5A2784412D5
:10B7CB00A65F12A4AE12A5A27F3F7E497DCD7C451C
:10B7DB0012A5A2784812A65F12A4AE12A2A012A2C2
:10B7EB009C785012A66B784C12A65F12A6148D553E
:10B7FB008E568F57785012A65F12A6148D598E5AFB
:04B80B008F5B786473
:10B80F00E557246AF608E556344CF608E555340436
:10B81F00F608E55B2458F608E55A34AEF608E43529
:03B82F0059F622A5
:1086240012A230128CB512A2347F66909841126C5B
:108634003D1286927F5A78C412866E12867678C668
:1086440012866E1286597F6578C812866E128676F7
:1086540078CA12866E7E2DE51B12C7567E33E51A44
:1086640012C7567E39E51902C756860408860302E6
:108674005BBC7E15E51C12C7567E1BE51B12C75654
:108684007E21E51A12C7567E27E51902C7567F5A7E
:108694007E01E53A12C66C7E0B9090A9E53B9302ED
:1086A400C769E6FF08E6FE08E6FD339217E45001C9
:1086B400F4FC12A68875130A75390112A88678D7B6
:1086C400E6C2E775F00A84F9303D02A9F012A688E3
:1086D4008913053912A85F30170A053912A87205E3
:1086E4003912A872A80302A66B12A230128CB5C26A
:1086F4003C7F5A7E031279D712869212D02610003C
:108704000810011510022080EFE53A146004153AB0
:108714008003753A3CD23C80DFE53AB43C05753AB7
:108724000180F2053A80EE7E031279D27E0B127933
:10873400D712869212D026100008100115100220BC
:1087440080EFE53BB40205753B158002153BD23C36
:1087540080DFE53BB41505753B0280F2053B80EEF6
:108764007E0B1279D27F5A78C412866E12867612E4
:0787740087DF12783678C49C
:10877B0012883778C612866E128659128811751CAC
:10878B000012783678C61288377F6578C812866EE5
:10879B001286761287DF12783678C812883778CA35
:1087AB0012866E128659128811751C001278367853
:1087BB00CA128837303C14E53B24F4500B78C9E6D9
:1087CB002410F618E63427F612883D12A2341273E1
:1087DB00B802D026C2247E15E51C127927F51CD2CF
:1087EB00247E1BE51B127927F51B1023E77E21E561
:1087FB001A127927F51A1023E67E27E51912792725
:10880B00F5191023E822C2247E2DE51B127927F5DA
:10881B001BD2247E33E51A127927F51A1023E77E33
:10882B0039E519127927F5191023E622ECF608EB36
:10883B00F6221290C178C8E6FE0886073395E0FD54
:10884B00FC12A5A27FE87E037D007C0012A8861295
:10885B00A5A278CAE6FE0886073395E0FDFC12A8B0
:10886B005F12A5A27F807E697D677CFF12A85FECFB
:10887B0012A5D912A5A27F3F7E807D0D7C1D12A46F
:10888B00AE12A5A27F3D7E407D007C0012A5A27892
:10889B00BC12A65F12A4AE12A5A27F3E7E807D0005
:1088AB007C0012A2A012A5A278BC12A65F12A4AEE5
:0988BB0012A5A27F3F7E807D0022
:1088C4007C0012A29C12A5A278B412A65F12A4AED8
:1088D40012A526783C12A66B7F407E807D007C002A
:1088E40012A5A2783C12A65F12A4AE12A70512A587
:1088F400A27F3F7EA87D007C0012A5A278B812A6B4
:108904005F12A4AE12A4AE12A5A27F407E007D0029
:108914007C0012A5A2783C12A65F12A4AE12A70591
:1089240012A5A27F3F7EC07D007C0012A4AE12A2DD
:10893400A012A5A278B812A65F12A4AE12A5A278BE
:108944003C12A65F12A2A0785412A66B12A6EF786E
:108954005812A66B12A5A212A4AE12A5A278C01238
:10896400A65F12A4AE784412A66B785412A65F12C6
:10897400A705783C12A66B12A5A212A4AE12A5A25A
:1089840078BC12A65F12A4AE783C12A66B7F3E7E22
:10899400C07D007C0012A5A2783C12A65F12A4AE92
:1089A40012A5A27F3F7E007D007C0012A2A012A52A
:1089B400A2783C12A65F12A4AE12A5A27F3F7E80CD
:1089C4007D007C0012A2A012A5A278B412A65F12A8
:1089D400A4AE787012A66B78C4E6FE0886073395B9
:1089E400E0FDFC12A5A27FE87E037D007C0012A8B6
:1089F4008612A5A278C6E6FE0886073395E0FDFC3C
:108A040012A85F12A5A27FE07E5E7DF87CFF12A80B
:108A14005FEC12A5D912A5A27F3F7E7F7DE57CC9BC
:058A240012A5A278700C
:108A290012A65F12A4AE12A526785012A66B7F3F3C
:108A39007EF07D007C0012A5A2783C12A65F12A4EC
:108A4900AE12A5A27F3F7EC07D007C0012A2A012BB
:108A5900A5A2783C12A65F12A4AE12A5A27F3F7E02
:108A6900807D007C0012A2A0783C12A66B78BC1213
:108A7900A65F12A5A27F3F7E807D007C0012A29C8A
:108A890012A5A2783C12A65F12A5A278B412A65F1D
:108A990012A4AE12A4AE784012A66B785412A65F47
:108AA90012A73D783C12A66B12A5A212A4AE787447
:108AB90012A66B7F417E107D007C0012A5A278C0B2
:108AC90012A65F12A4AE12A5A27F407E807D007C13
:108AD9000012A5A2784412A65F12A4AE12A5A27F25
:108AE900417E207D007C0012A29C12A5A27844122E
:108AF900A65F12A4AE12A5A27F407E407D007C0035
:108B090012A5A2787412A65F12A4AE12A5A27F4084
:108B19007EA07D007C0012A2A012A2A012A29C122B
:108B2900A5A2785012A65F12A4AE12A5A27850127F
:108B3900A65F12A4AE12A5A27F3D7E2A7DAA7CABB8
:108B490012A4AE12A5A27F3F7E007D007C0012A276
:108B59009C12A5A2783C12A65F12A5A2787012A653
:108B69005F12A4AE12A5A2784012A65F12A5261222
:108B7900A5A2785012A65F12A4AE12A5A27850122F
:108B8900A65F12A4AE12A4AE12A5A2785412A65FD3
:0C8B990012A29C12A5A27F4A7E517DD240
:108BA5007CCB12A4AE12A61478AC12A66B7F407EC5
:108BB500007D007C0012A5A2787412A65F12A4AEF7
:108BC50012A5A27F3F7E807D007C0012A2A012A587
:108BD500A2784412A65F12A2A012A5A2785012A6EE
:108BE5005F12A4AE12A5A2785012A65F12A4AE120F
:108BF500A5A2785012A65F12A4AE12A5A27F3E7E52
:108C05002A7DAA7CAB12A4AE12A5A2785012A65F4B
:108C150012A29C12A5A2785812A65F12A52612A52B
:108C2500A27F4A7E517DD27CCB12A4AE12A614122D
:108C3500A5A2AF3AEF3395E0FEFDFC12A5A27F4059
:108C45007E7E7D057C0012A88612A5A27F607E75BA
:108C55007D587CFF12A85F12A85F78B012A66B78CA
:108C6500AC751B64128C8C8F1C78B0751B67128CCD
:108C75008CE51C75F00AA42FFF249C50027F007818
:108C8500D7E654802FF62275390012A65F12A5A2E9
:108C95007F0A7E007D007C0012A932A81BE513F631
:108CA50008E512F608E511F6335004EFF404FF2247
:108CB500C23D78647BAC1286A6D23D78677BB01244
:108CC50086A61290C17F007EE47D577C0012A5A286
:108CD50078AC12A65F12A85F12A5A27F007E537D15
:0E8CE500077C0012A93212A5C185133B7F80C7
:108CF3007ECB7DA47C0012A5A278B012A65F12A839
:108D03005F12A5A27F407E7E7D057C0012A93212F0
:108D1300A5C1E513F56F04F53A85126E85116D85CE
:108D2300106C7F407E7E7D057C0012A5A2786C12BC
:108D3300A65F12A88612A5A27F607E0C7DA27C008E
:108D430012A5A278B012A65F12A85F12A872786C5F
:108D530012A66B78AC12A65FEC12A5D912A5A27F5E
:108D6300347E9C7D2B7C5F12A4AE785412A66B12CA
:108D7300A6EF785012A66B786C12A65FEC12A5D9F9
:108D830012A5A27F347E9C7D2B7C5F12A4AE12A51C
:108D9300A2785012A65F12A4AE784012A66B7F4051
:108DA3007E007D007C0012A5A2785412A65F12A457
:108DB300AE12A70512A5A27F3D7EC07D007C0012E6
:108DC300A5A278BC12A65F12A4AE12A5A27F3E7E16
:108DD300C07D007C0012A2A012A5A278BC12A65FDF
:108DE30012A4AE12A4AE12A5A27F3D7E407D007CEC
:108DF3000012A5A278BC12A65F12A4AE12A5A27F90
:108E03003E7E807D007C0012A2A012A5A278BC1237
:108E1300A65F12A4AE12A5A27F3F7E807D007C00D8
:108E230012A29C12A5A2785412A65F12A4AE12A29B
:108E33009C12A5A27F407E807D007C0012A5A278B3
:108E43005412A65F12A4AE12A70512A5A27F3D7EFF
:108E5300707D007C0012A5A278BC12A65F12A4AE9E
:108E630012A5A278BC12A65F12A4AE12A4AE12A2DF
:108E7300A012A5A278B412A65F12A4AE785812A6C7
:108E83006B785412A65F12A705783C12A66B785430
:108E930012A65F12A73D785412A66B783C12A65F08
:108EA30012A5A212A4AE12A5A278BC12A65F12A4A8
:108EB300AE783C12A66B7F3E7EC07D007C0012A57F
:108EC300A2783C12A65F12A4AE12A5A27F3F7E0039
:108ED3007D007C0012A2A012A5A2783C12A65F120C
:108EE300A4AE12A5A27F3F7E807D007C0012A2A0CB
:108EF30012A5A278B412A65F12A4AE787012A66B64
:108F0300785012A65F12A5A212A4AE12A5A278C031
:108F130012A65F12A4AE784412A66B785412A65F11
:108F230012A5A212A4AE787412A66B784012A65FA3
:108F330012A5A212A4AE783C12A66B7F407E807D60
:108F4300007C0012A5A2784412A65F12A4AE12A55B
:108F5300A27F417E107D007C0012A2A012A5A27800
:108F63004412A65F12A4AE12A5A2787412A65F12D1
:108F7300A5A27F407EA07D007C0012A29C12A2A02D
:108F830012A5A2783C12A65F12A4AE12A5A27F3D41
:108F93007E2A7DAA7CAB12A4AE12A5A27F3F7E00DF
:108FA3007D007C0012A2A012A5A2785412A65F1223
:108FB300A5A2787012A65F12A4AE12A5A2783C12E5
:108FC300A65F12A4AE12A4AE12A5A2785812A65F91
:108FD30012A2A012A5A27F3F7E7F7DE57CC912A4C9
:018FE300AEDF
:108FE40012A5A27F4B7E187D967C8012A2A012A6A9
:108FF4001412A5A27FE87E037D007C0012A9321220
:10900400A5C178C8A61208A61308A60608A607785C
:109014007412A65F12A5A27F3F7E807D007C0012A1
:10902400A29C12A5A2784412A65F12A2A012A5A225
:109034007F3E7E2A7DAA7CAB12A4AE12A5A2784004
:1090440012A65F12A4AE12A5A2783C12A65F12A4C7
:10905400AE12A5A2784012A65F12A2A012A5A27F0A
:109064003F7E7F7DE57CC912A5A2787012A65F12AF
:10907400A4AE12A4AE12A5A27F487EF47D247C0087
:1090840012A2A012A61412A5A27FE87E037D007C82
:109094000012A93212A5C178C4A61208A61308A604
:1090A4000608A607223F3F4344454647484A4B4CDF
:1090B4004D4E5051525354555657583F3FE4F5398D
:1090C400F5A79090D5791078B4E493F6A308D9F96C
:1090D4002232A5C24A4A19DC3A885CDB3BFFD6DC63
:0190E4003B50
:10A23000D2D58002C2D575A70490040078107F0B98
:10A2400012A25C78267F0512A25C783C7F2212A2C3
:10A250005C786A7F0F12A25C75A7002230D506E6F3
:10A26000F008DFFB22E0F608DFFB22D2D58002C235
:10A27000D575A7049006FA78737F0612A25C75A7BD
:10A280000022DA0CD902800BD906303701B3500511
:10A2900002A40F923702A3FBD9F680F9D2368002CE
:10A2A000C23612A440303606C86002B237C89236B1
:10A2B000DAD0D9E4B8000A12A487A236923702A3F2
:10A2C000E460FBB51300400F12A487A23692F7A2F8
:10A2D000379236A2F79237C398F40424E740DF247C
:10A2E00019AD29AC28AB277A00C394084008CDCC1F
:10A2F000CBCAE4CD80F424086010F9C3ED13FDEC63
:10A3000013FCEB13FBEA13FAD9F1A236303701B391
:10A3100040308A17E5102BF518E5113CF519E512C8
:10A320003DF51A501A13F51AE51913F519E5181326
:10A33000F518E51713F5170513E513700205140258
:03A34000A39AE4F9
:10A34300C39AF517E5109BF518E5119CF519E5126D
:10A353009DF51A500DB237C378177F04E496F608BB
:10A36300DFFA7A047019E513C39408F51350021544
:10A3730014E4C517C518C519F51ADAE802A43B2079
:10A38300E7BAE5137002151415137817C37F04E6B3
:10A3930033F608DFFA80E8E51A20E7137817C37F5E
:10A3A30004E633F608DFFAE513700215141513E516
:10A3B300173378187F03E63400F6500E08DFF7757D
:10A3C3001A800513E51370020514E51420E7547091
:10A3D30027E513604E046020851A1285191185182C
:10A3E300105326F0AC10AD11A237E51313FFE5129D
:10A3F30092E7FEA81302A5C1E4F512F511F510F5D5
:10A40300147513FF5326F043260580D8E5FFF51294
:10A41300F511F510751400F513D2375326F04326C2
:10A423000980C15326F0432603E4F512F511F51014
:10A43300F514F513C23780AC5326F080EC79017A1A
:10A44300018512F0E513A2F7339237751400F51363
:10A453006002D2F785F012A813B8FF0809E512C20B
:01A46300E711
:10A464006001098C278D288EF0A2F7EF3304700A5F
:10A474000AC2F705F00AD5F0011A146002D2F78572
:10A48400F02922C88813C512C529C512C511C528CB
:10A49400C511C510C527C51022DA03B8000302A4EC
:10A4A4000FD9028002D9F702A3FB12A4403037016E
:10A4B400B392377004D9E78005DADEB8000302A44A
:10A4C4003BD9E2C3947E500215142513F5135002B0
:10A4D40005147815760008B81BFA78277915E6086C
:10A4E400FAE8FC78108AF0E608A427F709E5F037C3
:10A4F400F7500989F00907E760FBA9F0B813E619DA
:10A5040019ECF8B82AD802A39A02A426B8FFFA02D2
:10A51400A40FD9FB02A3FBDAF6B800F002A43B12A5
:10A52400A67712A440303701B392377007D9E3B845
:10A5340000E280DBDAE1B8000280E1D9D5C8C39833
:10A5440050021514247F50020514F513781A76006E
:10A554007A1A7B80C3E5109527E5119528E51295B5
:10A56400294016C3E5109527F510E5119528F51136
:09A57400E5129529F512E64BF6FB
:10A57D00DA0302A39AEB03FB30E703187600C3E579
:10A58D001033F510E51133F511E51233F51240CA0C
:10A59D0030E7DD80B6E53905396010D0F0D0E0C088
:10A5AD0010C011C012C013C0E0C0F08F138E128DF9
:10A5BD00118C1022E539146010D0F0D0E0D013D0FA
:10A5CD0012D011D010C0E0C0F01539227920800CC6
:10A5DD007910800479087D007E007F003392D5507C
:10A5ED000312A651EC33400FEF33FFEE33FEED3384
:10A5FD00FDEC33FCD9EE22EECCF5F0747E29A2D51C
:10A60D0013FF92F7AEF022EF8EF0A2F7D2F733924E
:10A61D00D5C3947F5006E4FFFEFDFC229420400438
:10A62D0074FF80F304CCFEE4FFFAE5F0CC6012C3B6
:10A63D00CC13CCCD13CDCE13CECF13CF0450EEDA39
:10A64D00EC30D5D7C3E49FFFE49EFEE49DFDE49C72
:03A65D00FC22E6F6
:10A66000FC08E6FD08E6FE08E6FF22ECF608EDF63B
:10A6700008EEF608EFF622CFC513CFCEC512CECD29
:10A68000C511CDCCC510CC22E4F513F512F511F5AA
:10A690001022E493FCA3E493FDA3E493FEA3E493CC
:10A6A000FFA322C0E012A5A212A4AE12A6D612A643
:10A6B00092D0E0C0E012A5A212A6CD12A4AE12A5BF
:10A6C000A212A69212A2A0D0E0D5E0E722AC48AD3B
:10A6D00049AE4AAF4B228C488D498E4A8F4B22742B
:10A6E000FF7809FFFEFDFCE52654F048F52622120E
:10A6F000A79604A2E1927F1420E01590A817740495
:10A7000012A6A3802912A79630E102B27F20E0EBC7
:10A710008C4C8D4D8E4E8F4F90A82B740412A6A397
:10A7200012A5A2AC4CAD4DAE4EAF4F12A4AE307FD1
:10A7300004EF6480FFEE33EF337001FF2212A7961F
:10A74000C0E08C4C8D4D8E4E8F4F90A84F740312ED
:10A75000A6A312A5A2AC4CAD4DAE4EAF4F12A4AE07
:01A76000EC0C
:10A76100C54CFCEDC54DFDEEC54EFEEFC54FFF904E
:10A77100A83F740312A6A3D08212A5A2AC4CAD4D82
:10A78100AE4EAF4FE58230E00712A526B27F809D25
:10A7910012A5238098EE33EF3324605007D0E0D028
:10A7A100E002A6DFEFA2E7547F927FFF12A5A27C11
:10A7B100837DF97E227F3E12A4AEEE33EF332481F6
:10A7C100501012A5A212A61412A5D9EFB2E7FF12DA
:10A7D100A2A0EE33EF33602A2403F8C313FFEE92F5
:10A7E100E7FEE82481E4501A12A5A212A614EF0490
:10A7F100C2E0FCF58212A5E1EFB2E7FF12A2A0E5EB
:10A801008203FAEE33EF33600B148FF0A2F713FFDC
:10A81100EE92E7FEEA2283FA703AE4E9AABCF8E094
:10A82100813EE6E99DBF0000803F1A3C28396669F8
:10A8310099BBE335A33DE75D25BFDB0FC93FCCDB0A
:10A841008D41EE3649C43F91C9453DF8B0C5000080
:10A85100803F34F517C373FA2F45DDFD0AC6EF2596
:10A8610013FFEE3512FEED3511FDEC3510FC02A59E
:10A87100C1C3EF9513FFEE9512FEED9511FDEC9519
:10A8810010FC02A5C1EFF88513F0A4FFE513C5F094
:0AA89100CEF9A42EFEE435F0CDFA56
:10A89B0088F0E512A42EFEED35F0FDE433CC8513E4
:10A8AB00F0A42CFCE5128AF0A42CFCE51189F0A491
:10A8BB002CFCE51088F0A42CFC89F0E512A42DFDEE
:10A8CB00EC35F0FCE51188F0A42DFDEC35F0FC8A9D
:10A8DB00F0E513A42DFDEC35F0FC02A5C1E4CCF89A
:10A8EB00E4CDF9E4CEFAE4CFFB75F020C3E51333E6
:10A8FB00F513E51233F512E51133F511E51033F5C8
:10A90B0010EF33FFEE33FEED33FDEC33FCEF9BEE3C
:10A91B009AED99EC98400CFCEF9BFFEE9AFEED99AB
:10A92B00FD0513D5F0C622C2D5EC30E705B2D51222
:10A93B00A651E51030E70DB2D512A95512A8E812B1
:10A94B00A651800312A8E830D515C3E49513F5136F
:10A95B00E49512F512E49511F511E49510F510221A
:109A1300E57124885002D219125F458E4712C47C27
:109A23001286041262EE305E0F12628C127D2912CE
:109A330061CA12B37B123D111234571242DA103647
:109A430029201F1C301219E4129B99129BAE129C01
:109A5300B0129CD2305103029D5C12A02D205109FB
:109A6300C251E4F552F545F5442275A70075830705
:109A7300E559C454F0F582E0F538A3E0F518A3A343
:109A8300A3E0F51E74FF129B99125F458E1C8F1B7A
:109A93007510DF751100E51164B47006129B6475CF
:109AA3001110129B314028AE1CAF1B125FCB20322A
:109AB3001EAC03AB027A0C125BF4ED701275A700B7
:109AC300758304851182ECF00583E510F00511D54B
:109AD30010C4129B6475C70375C6E075A70490058F
:109AE300007F04129B1FDFFB75A7001225DF1262A4
:109AF3008CE4F5A7F8F559758307E8C4F582E065AA
:109B0300387011A3E06518700BA3A3A3E0651E7062
:109B13000388592208C3E5589850DC22E0F5BCE0DD
:109B2300F5BDE0F5BEE0F5BF1248EE05C622E5102F
:109B330075F004A4F5C685F0C775B901E5BC3340DB
:0B9B43001F05C605C675B90185BE648C
:109B4E0085BF6505C675B90185BC6685BD6785BED1
:109B5E006885BF69C322E51124FE502E75A7007FCC
:109B6E0010AE111E7583048E82E0FD1582E0CDB518
:109B7E0005005012F00582CDF00583E0FD1582E060
:109B8E00CDF00582CDF0DEDCDFD72275A754900430
:109B9E000005A79005007FB4F0F0DFFC75A700224A
:109BAE0012B1C7C2517B077AFFE4FFF5A7900400FC
:109BBE00129C94ED244C4035EC603075A7008D82DC
:109BCE0005A7129C5A7583058D82E02410401CF067
:109BDE0005A7E02CF0500505A7E004F0BA000CBB79
:109BEE000009D251EF24DC50027F23DFC3EA600567
:109BFE00129C0D8006EB6003129C4575A700223067
:109C0E00E0047553082230E1047553182230E20443
:109C1E007553282230E3047553382230E40475530B
:109C2E00482230E5047553582230E60475536822F5
:109C3E0030E7037553782230E0047553882230E103
:109C4E00047553982230E2037553AA22ED54F0C4E2
:109C5E002323909C64735302FE225302FD2253026F
:069C6E00FB225302F72265
:109C74005302EF225302DF225302BF2253027F22F8
:109C84005303FE225303FD225303FB225303FB22FF
:109C940012B0D912AF68E4F5F7C2B2C2B2ADF7F5AB
:109CA400F7C2B2C2B2ACF7D2B2C220229005007899
:109CB400B4E06015FD54F0C4CD7C00540FFE158350
:109CC400E0FF125CF2EFF005830582D8E42275838D
:109CD4000478FF088882E060FAF5D38812E512243C
:109CE4004C50012285D3D288D4881279FF0512E51D
:109CF4001260F00908E875F0B484A8F08882E06086
:109D0400ECF5D3B9000280D5B9230050D0C395D265
:109D140092D15002F40409FEE4FFFCAD01125CFF91
:109D24007401FA25D475F0B484A8F0AC06AB07121C
:109D34005BE6EB30E7010CE5D22C30D1029C9C8829
:109D440082F00AEAB501DCE512244C50012285D3E5
:109D5400D28512D4A8128093900400129E1B8C0604
:109D64008B05129E1BE4FFF512F5118C148B13C3A3
:0E9D7400ED9BF9EE9CFA4012E51199E5129A6A
:109D8200500A8C148B138A1289118F528F82E0F938
:109D9200C3ED99FDEE9400FEE582245A5002244C54
:109DA20075F0B48485F082E0FA2DFDEE3400FEEB0E
:109DB2009AFBEC9400FCE92BFBEC3400FC0FBFB4E3
:109DC200B0E55224D3400224B4F552C3E51333FB69
:109DD200E51433FCE511FE2BFBE512FF3CFC125DA2
:109DE20054E9F8909E2D93F511FDEBF513FFECF578
:109DF20014FE7C00125CF28F44E8909F2D93FAAB24
:109E020013AC14125C1DAF03AE04AD117C00125CE6
:109E1200F2EF7002F552F545227C007B007F5AE09A
:109E22002BFBEC3400FC0582DFF522B4B4B4B4B4ED
:109E3200B4B4B4B4B4B4B4B4B4B4B4B4B4B3B3B3E3
:109E4200B3B3B3B3B3B3B3B3B3B3B2B2B2B2B2B2E6
:109E5200B2B2B2B1B1B1B1B1B1B1B0B0B0B0B0B0F3
:109E6200B0AFAFAFAFAFAEAEAEAEAEAEADADADAD0D
:109E7200ADACACACACACABABABABAAAAAAAAA9A931
:109E8200A9A9A9A8A8A8A8A7A7A7A7A6A6A6A5A55D
:109E9200A5A5A4A4A4A4A3A3A3A2A2A2A2A1A1A192
:109EA200A0A0A0A09F9F9F9E9E9E9D9D9D9D9C9CCD
:109EB2009C9B9B9B9A9A9A9999999998989897970B
:109EC200979696969595959494949393939292924D
:109ED200919191919090908F8F8F8E8E8E8D8D8D8E
:109EE2008C8C8C8B8B8B8A8A8A89898988888887D3
:109EF2008787868686858585848484838383828218
:109F0200828181818080807F7F7F7E7E7E7E7D7D5B
:109F12007D7C7C7C7B7B7B7A7A7A7979797878789C
:109F22007777777676767575757474000203050611
:109F320008090B0C0E101113141617191A1C1D1FE9
:109F42002122242527282A2B2D2E3031333436374F
:109F5200393A3C3D3F404243454648494B4C4E4FBF
:109F6200505253555658595A5C5D5F60616364663E
:109F720067686A6B6C6E6F707273747677787A7BCF
:109F82007C7E7F80818384858688898A8B8D8E8F73
:109F92009091929495969798999B9C9D9E9FA0A133
:109FA200A2A4A5A6A7A8A9AAABACADAEAFB0B1B208
:109FB200B3B4B5B6B7B8B9BABBBCBDBEBFC0C0C1F9
:109FC200C2C3C4C5C6C7C7C8C9CACBCCCCCDCECF05
:109FD200D0D0D1D2D3D4D4D5D6D7D7D8D9DADADB28
:109FE200DCDCDDDEDEDFE0E0E1E2E2E3E4E4E5E565
:109FF200E6E7E7E8E8E9EAEAEBEBECECEDEEEEEFB8
:10A00200EFF0F0F1F1F2F2F3F3F4F4F4F5F5F6F621
:10A01200F7F7F8F8F8F9F9FAFAFAFBFBFBFCFCFDA2
:10A02200FDFDFEFEFEFEFFFFFFFFFFC251E4F54411
:10A03200F814FB900400A9007C0FC2D112A148E8D9
:10A042002405F8B8B4F08B13E5122403FA244C501B
:10A0520001FABBFF012275112C8A1912A17F8F16FA
:10A06200203D12AA1975112312A17F8F15751600B2
:10A07200303DE2801175112312A127751500303D84
:02A0820005E8EF
:10A084002F13F51575111212A127751400303D0513
:10A09400E82F13F514EA2404F552244C5002F55227
:10A0A400E4F51AF51BF51CE516600AFB7A00AF13FC
:10A0B4007EFF12A0EDE515600AFB7A4FAF137EFF19
:10A0C40012A0EDE516600DFB7A00E5146006FF7E34
:10A0D400CF12A0EDAE1CAF1B7C00AD1A125CF28F48
:10A0E40045EF2513F544D25122EFF5F0A4FCADF071
:10A0F400EBF5F0A49CFCE5F09DFDEB8AF0A4FAAB33
:10A10400F0EF8EF0A49AF8E5F09BF9E833F8E93320
:10A11400F97B00125D98051AE51B2BF51BE4351C31
:10A12400F51C22EA2511F9244C5001F9C2D112A1DF
:10A1340046303D428F00C3EA9511F9500324B4F927
:10A14400D2D17C09E4FDFEFF8982E060062FFFE4A2
:10A154003EFE0D09B9B4027900DCEDED20D118F50D
:10A164001E24FE923D500F125CFFEFB50300500613
:0EA17400851E1FFB881222F51D80E612A12712
:10A18200203D43740212A21E12A127203D387404FE
:10A1920012A22612A127203D2D740612A21E12A180
:10A1A20027203D22740812A22612A127203D1774EF
:10A1B2000A12A21E12A127203D0C740C12A2261212
:10A1C200A127203D0122C3E89F605088148F158A81
:10A1D2001640081ABAFF0A7AB380060ABAB4027A9B
:10A1E2000012A127303D34C3E89FF9602EC3E51465
:10A1F2009515FB6930E7D4E930E703F404F9EB3055
:10A20200E702F404C3995002AA16E5142515C82FD3
:10A2120028FFE4FC33FE7D04125CF2222AFA244C6D
:0EA222005001FA22C3CA9AFA500324B4FA2259
:10AF3600C2B212D0C7D2B275F83022C2B2F5F7C289
:10AF4600B2C2B2D2B222D220C2B2F5F7C2B2C2B2F5
:10AF5600856CF7C2B2C2B2856BF7C2B2C2B2856A5D
:10AF6600F722D220C2B275F703C2B2C2B2856FF71A
:10AF7600C2B2C2B2856EF7C2B2C2B2856DF722D234
:10AF86002012AFB9740612AF41740212AF4C8FF79C
:10AF9600C2B2C2B2D2B2C22022D21412099B125A33
:10AFA600F31248EED22012AFB9740612AF4174C73D
:10AFB60012AF4112AFBF40FB22C2B275F705C2B253
:10AFC600C2B2C2B2C2B275F705C2B2C2B2C2B2C290
:10AFD600B2E5F7D2B2A2E02212099B85BF6C85BE0C
:10AFE6006B756A00E56B7017E56A7013D22012AFB5
:10AFF600B9740612AF4174D812AF4CD2B2D21FC286
:10B006002022E54B0475F03C8485F04B12B2F385A3
:10B016002E72E55F030354C0F8E55E543F28F57CC5
:10B026003055012212B06312AFBF40F7E54C60F312
:10B0360012AFB912B07A12B04480F112AFB9C21F82
:10B04600D220740612AF41740212AF4C787086F7A4
:10B0560008B880FAD2B2C22012B09780877870758D
:10B06600A704758304E54CC4F5827F10E6F0DFFC87
:04B07600054C8019EC
:10B07A00787075A704758304154CE54C30E701E434
:10B08A00C4F5827F10E0F6DFFC75A7002274102554
:10B09A006A54F0F56AE4356BF56BE4356C540FF5D8
:10B0AA006C22E54B75F010A4256A54F0F56AE5F0B8
:10B0BA0080E4E56A24F054F0F56AE56B34FFF56B39
:10B0CA00E56C34FF80D7E56A24FF80ECC380EBE5AA
:10B0DA006D24F054F0F56DE56E34FFF56EE56F34CE
:10B0EA00FF540FF56F2275A7047583048F82787059
:10B0FA00E6F008B880FA75A7002275A7049004B490
:10B10A007F20E4F0DFFD80EE12B16E12B19AC22DFB
:10B11A00C254C255E57F7002D255147002D254E56A
:10B12A004A30E00122B4061E20540F12B0BC12B2FB
:10B13A003E12B2D212B30A02B41A1279F67E04127D
:10B14A00D0BF754A012220550F12B09712B2B11220
:10B15A00B2F312B21702B3ED1279F67E0412D0BF1F
:10B16A00754A0522740312AF4C7870E4F5F7C2B23F
:10B17A00C2B2A6F708B880F3D2B2C2202274031270
:10B18A00AF4CE4F5F7C2B2C2B2E5F7D2B2C220229E
:10B19A00E575F8541F30E40244E0F57585722EA275
:07B1AA00779226E57C543F7B
:10B1B10030E50244C0F55EE57C54C02323F55FE52C
:10B1C1007F1414F55122856C6F856B6E856A6D2233
:10B1D100856F6C856E6B856D6A22E4FEFF74077561
:10B1E100A704F5838E8274FFF0DFFD75A70022743A
:10B1F100067E007FB012B1E0E4F55AF55B2275A737
:10B2010004758306E55A600A75F00A84E5F0700258
:10B21100740AC4F58222307720E55A2402400205DF
:10B221005A12B1FFE55AF0E573F0E574F0E575F0F7
:10B23100E576F0E577F0E578F075A700223077F94B
:10B2410012B1FF7F1074FFF0DFFDE55A24F55003C2
:10B2510012B269155AE55AB4FF02055AC3E55A9567
:10B261005B50D6755B0080D112B1C77F0A056D05B1
:10B271006D12AF68E4F5F7C2B2C2B2E5F7D2B2C25D
:10B281002030E704DF02800512B0D980E0056D129D
:10B29100AF6812B1FFE55A24F6F07F06E4F5F7C274
:10B2A100B2C2B2E5F7F0DFF4D2B2C22075A7002234
:10B2B100053FE53FB43C17753F00053EE53EB43C14
:10B2C1000D753E00053DE53DB41803753D00024591
:10B2D100B0153FE53FB4FF17753F3B153EE53EB462
:02B2E100FF0D5F
:10B2E300753E3B153DE53DB4FF03753D170245B083
:10B2F3000542E542B43C0F7542000541E541B43CCB
:10B30300057541000540221542E542B4FF0F754221
:10B313003B1541E541B4FF0575413B154022AC4067
:10B32300AB41A842EC75F03CA42BFBE435F0FC7A6E
:10B333003C125BE6EB28FBE43CFC22AC3DAB3EA8B5
:10B343003F80E178AE8604AB3EE53FC313F880113E
:10B35300120991ACBF53041FE5BE75F005A4FB7839
:10B3630000EC75F03CA42BFBE435F0FC7A1E125B79
:10B37300E6EB28FBE43CFC2212B353AE04AD03120C
:10B38300B3468C148B1312096EE5BFFF24F65002EB
:10B393007F01E5BE75F096A4AAF0F9C3ED9513FB02
:10B3A300EE9514FC924E4B701120110E30480B7524
:10B3B300364B3003037536FFD22E304E02DF1F7A31
:10B3C30002125BE675A7009004EEECF0A3EBF0C36A
:10B3D300E5BF9F04BF0102D2E79005CBF022ED2920
:10B3E300FDEE3AFE80B520740122C3E5709557FF48
:02B3F30024FD37
:10B3F5005021EF24EB400A78BD06B60016180680EA
:10B4050012EF2402400DEF2414500878BB06B60055
:10B41500021806802BC3E5709557FF24FD5021EFD8
:10B4250024EB400A78BB16B6FF1618168012EF24D7
:10B4350002400DEF2414500878BD16B6FF02181609
:04B445008570572295
:10D0AC0012D0B512D0B512D0B57E0480067E0280A7
:10D0BC00027E017F0080087F6480027F017E00EF8A
:10D0CC004E6012E4FD0D1D0DEDC394AD40F7EF1F46
:10D0DC0070ED1E80EA22753500C200C201C2022228
:10D1D200F5D8D2DCE5F520E7FBE5DA540FFEAFD94E
:04D1E20075D80022DA
:10CE08007F767E069090FA126C0C740412D1D27C54
:10CE1800007D52125CF2EFF875F00A84C0F07F765C
:10CE28007E2312C7567E29742E12C7697E2ED0E043
:10CE380012C7567E35745612C7697F6B7E1190CE25
:10CE48007112C797E824E04001220423F824E75030
:10CE580002781812CE61D8FB227F6CE82411FE7983
:10CE68000512D12B0E0FD9F922071DFFFFFFE08015
:10CE7800000020C0000038E0000008F0000038F88A
:07CE8800000020FFFFFFE0A6
:10CF0D0012CF3530E6022409540F75F00AA4F51539
:10CF1D0012CF3530E6022409540F25152212CF35D4
:10CF2D00540F2275F000800875F044800375F007EA
:10CF3D00E4206D09D5E0FAD5F0F7D24C229247C224
:10CF4D00ACE54F623885504FA26E926D859950C2F7
:10CF5D006FD2ACC24CA2472212CF6FC4FA12CF6F60
:10CF6D002A2212CF3520E603540F2254072409221A
:10CD7600E612CD7D18E608FAC412CD83EA540F44B4
:10CD860030F924C6E950112407800D75F00A84C0D5
:10CD9600F012CD9CD0E0443030530975F00085E0A8
:10CDA600E0D5F0FA3099FDC299F599623822E53856
:10CDB60080F2E53812CD7D800812CD9EE53812CD81
:10CDC6009E740D12CD9E740A80CE744012CD9E7450
:10CDD6004080C5742C80C1742E80BD12CDF9E91235
:10CDE600CDAA800312CDF9E812CDAAE53812CDAA54
:10CDF600024358124358800312437074407538003A
:02CE0600809614
:10D1F80085A0835383FE438380858384F0758400F0
:01D208002203
:10CC240074A212D1F874A112D1F874A612D1F874B6
:10CC3400A412D1F874C012D1F8742512D1F812CC10
:10CC4400B475C70375C6FC75B90112A96B740812D3
:10CC5400D1D2EE75F020A4FEEF54F80303032E2482
:10CC640092C313FE24EA50027E16EE90CC9D9325C7
:10CC7400BCFE24E6501F24E8401B748112D1F8EE58
:10CC840012D1F812CCC1744012D1F8742F12D1F819
:10CC940074AF02D1F87E2680E1F7F7F8F8F9FAFBD1
:10CCA400FCFDFEFF00000000010102020203030379
:10CCB400A8BCA9BDAABEABBFACC7ADC62288BC89FF
:0ACCC400BD8ABE8BBF8CC78DC6224F
:10D02600D21AC006C007C0E075A7019000007EB7FF
:10D0360075A700EE12D1F8741012D1F8740412D14B
:10D04600F885A08343838185838475A7517F80E01B
:10D05600F0DFFC1EBEAFD9E4F5A7F584D0E0D0071B
:05D06600D006C21A22F1
:10D1E60075A711900000E4C583F0C58330E2F8F519
:02D1F600A7226E
:10D12B00EF20E723EE20E71F20E61C05A7C45403DE
:10D13B00F583EE5408C42FF582EE5407240983F5CA
:10D14B00F0E045F0F005A722804020100804020112
:10D15B00EF20E723EE20E71F20E61C05A7C45403AE
:10D16B00F583EE5408C42FF582EE5407240983F59A
:10D17B00F0E055F0F005A7227FBFDFEFF7FBFDFED8
:10C71600FDA42582F582E5F03583F583ED22906848
:10C726005A7A0475F00512C7167D0580607A058071
:10C73600027A04547FC0E0C083C082C394205001B3
:10C74600E490680A12C72980309069687A058005E6
:10C75600906A257A0675F00712C7167D07802E7A2D
:10C766000580027A06547FC0E0C083C082C394204D
:10C776005001E49069B512C75BD082D083D0E02225
:10C7860090678875F00A12C7167D0A7A07C2D180AB
:10C7960002D2D1C0A7C082C083C007C006C0E030A5
:10C7A600D10975A704E493FDE493FAEEFB75A7049B
:10C7B600EBFEEAFC7901D9067908E493F5D4E5D4D1
:10C7C60023F5D420E01612D15B0EDCEA0FDDE1D0B2
:10C7D600E0D006D007D083D082D0A72212D12B80FA
:10C7E600E89066C875F00E12C7167D0E7A0812C755
:10C7F6009390677075F00212C716E493FDE4A39355
:10C80600FACE2408CE7C0812C8147C06AD02ED23AD
:10C81600FD20E00712D15B0FDCF42212D12B80F74A
:10C60100F5D2C2D58036F5D2D2D58030F5D224F616
:10C6110050090E0E24A650030E0E0EE5D2F5D2756A
:10C62100F0648485F0D3C2D57009D2D5742012C7C5
:10C6310069800312C756CE2406CEE5D375F00A846D
:10C6410085F0D3700A30D507742012C769800312B0
:10C65100C756CE2406CEE5D312C756E5D222F5D26F
:10C6610075F0648485F0D3C2D58022F5D2C2D5801D
:10C6710025F5D2D2D5801FF5D275F0648485F0D32B
:10C68100C2D57009D2D5742012C769800312C74F71
:10C69100CE2405CEE5D375F00A8485F0D3700A3037
:10C6A100D507742012C769800312C74FCE2405CE67
:10C6B100E5D312C74FE5D222F5D2C2D58035F5D2E6
:10C6C100D2D5802F30E70DF404C0E0742D12C737A6
:10C6D1000E0ED0E0F5D275F0648485F0D3C2D5702A
:10C6E10009D2D5742012C737800312C724CE24047F
:10C6F100CEE5D375F00A8485F0D3700A30D507747E
:10C701002012C737800312C724CE2404CEE5D312EA
:05C71100C724E5D2225F
:106BFA007E00800E7405FEF51EE4FFF51DF51F20CC
:106C0A003C3375A700E493700122A3B40204051D66
:106C1A008003B4010A051FEF2409FFAE1E80E612A5
:106C2A00C7697D06B440027D03B421027D02EE2DC0
:106C3A00FE80D27E0075A700E493700122A3B402FD
:106C4A0004051D8003B4010F051FEF2407FFAE1EC4
:106C5A0080E612C7338008B45B0050F612C7370EBD
:106C6A00B4210280D30EB4400280CDB42C0280C875
:106C7A000E0EB45F0280C1B45B0040BC0E0E80B839
:106C8A00E60812C769EE2406FED513F4229090FF97
:106C9A00307409909103307303909108026C0C755B
:106CAA00F019D5E0FDD5F0FA12431E12CDD0744F7B
:106CBA0012CE03744B12CDBFC322C250126D0812FA
:106CCA00431ED2AC12CF30304C1212CF30304C0CA3
:106CDA0012CF30304C06D250C2ACD322B440E512A7
:106CEA00CF35B4400312CF35B44FED12CF35B44B84
:106CFA00E712CF3512CF3512CF35C2ACC32230538B
:106D0A000975F008D5E0FDD5F0FA227F0575F0196E
:106D1A00D5E0FDD5F0FA12431E12CDD0745712CE2B
:106D2A0003745012CD9E748112CD9EE56312CD9EDE
:076D3A00E56212CD9E78D046
:106D4100E612CD9E08B8D7F8E6F8795F30E7027908
:106D51002FE912CD9E12CD9E12CD9E12CD9E74585A
:106D610012CD9E744312CD9EE412CD9EE8C2E7750A
:106D7100F00A84C425F012CD9E7864E612CD9E08F7
:106D8100B869F8E612CDBF126CC4400122DF02805F
:106D91000A20508B75F0008080D250C2ACD32212F1
:106DA1006D08C25012431ED2AC2002EF12CF302028
:106DB1004CE7B440F412CF35B4400312CF35B45789
:106DC100DAF53812CF35B450D212CF3512CF35F5AE
:106DD1006312CF35F56278D012CF35F924A0500374
:106DE10053015FE924E04002795FA60108B8D8E8C1
:106DF100780612CF35D8FB12CF35FC53040FC4549B
:106E01000F75F00AA42CFC249C50027C0078D786D4
:106E110001E4B92F02D2E72CF6786412CF35F608D7
:106E2100B86AF812CF35E5386003026D9C12CF3590
:106E310012CF35C2ACC3229096EE80039093947F1B
:106E410020126C3D12D02602D0BD753400C26B12E7
:106E51006F0012D0BD127272E5166003126E6302EA
:106E610002571274D61218E212D026100020100117
:106E71000280F81272DD50131218ED126E381000F4
:106E81000D10010280F812188F80D712705E22C295
:036E91006BD2279A
:106E940075480A1225D37534001273ACC26A122FD6
:106EA4001F106A0512024880ED1202481272041281
:106EB400735C1273B81274D61218E212D026100042
:106EC4003810010280F81272DD501BE96515601854
:106ED4001218ED126E3812D0B510001D1001028088
:106EE400F812188F80C3D26B1273887516078559F0
:106EF4001712264C753500809D02025712727212C9
:106F04006F221273B87F19126F3C90971B7E121276
:106F14006C3F7E23E51602C6D590981480EF786204
:106F2400E4126F3378D0745F126F3318E4F6227F63
:106F340008F608DFFC227F7B7E007810742012C7DD
:106F440037CE2404FED8F5227F197E08126C3F7ECA
:106F54002890937630530390937B026C3FC26B125C
:106F64006F22126F6C020257C2511273B8909713BA
:106F7400126F4C1218B51272727F20126F0B12D05E
:106F840026E516700512D0B2803675A6FF3051037F
:106F9400126CB212431ED2AC200025306DFA126D71
:106FA400A3400C1272DD401112705ED25180BB10EE
:106FB4005003126E3DC25180D1D251126E3880CA34
:106FC400C2AC22D22775480A1225D3753400C26B8D
:106FD4001273ACC26A122F1F106A0512024880EBAA
:106FE40012024812720412735C1273B8126FF850D2
:106FF400DA02025790938F126F4C1218C712D026E0
:04700400C3100013A2
:1070080010010510020E80F4126D15400122126E57
:107018003D80DDD3C2AC22D227C26B75480A122547
:10702800D37534001273ACC26A122F1F106A05128E
:10703800024880EDD26B12720412735C12722C75C6
:10704800B901E5BCB2E7F5BC1248EE7516078559DB
:107058001712264C80CBD26B127388127243E51735
:1070680075F01084240AF54824E8500375480A127C
:1070780025DF85585922D22075320012B1DB75A759
:107088000490070075150012722C75B901E5BC2033
:10709800E705E515F0801004600D6482600975BC91
:1070A800FF75B90575B9020515E515242050D8E511
:1070B8008224FE4003027159A882187F0075A70038
:1070C8007583078882E0FE75F004A41271D7A9BC05
:1070D800AABDABBEACBF1582E0FD75F004A4127169
:1070E800D7C3E995BC404C7052EA95BD4045704BFA
:1070F800EB95BE403E7044EC95BF4037703DEE7551
:10710800F004A4041271D7A9BCAABDABBEACBFEDF4
:1071180075F004A4041271D7C3E995BC4015701B1F
:10712800EA95BD400E7014EB95BE4007700DEC95C6
:09713800BF5008EEF00582EDF0F5
:107141001582E5826009C3EF958250030270CD0F6D
:10715100C3E89F40030270C575A70490070075C777
:107161000375C6A8E0F5BCE0F5BDE0F5BEE0F5BFEE
:1071710075B90575B90205C6E58224204006E5C644
:10718100242050E00875C70375C68075B901E5BCB8
:107191001271C1F5BCE5BD1271C1F5BDE5BE12713B
:1071A100C1F5BEE5BF1271C1F5BF75B90205C6E5EE
:1071B100C6245850D6E5320470FB75A700C22022C0
:1071C100B4FF0122F975A704900700E58268600504
:1071D100E06970F7E922F5C685F0C775B901E5BC2C
:1071E100645F700375BC27E5BD645F700375BD27DF
:1071F100E5BE645F700375BE27E5BF645F7003750C
:10720100BF272275C703E54875F004A42480F5C69D
:10721100E55975F00484A8F00825C6F5C675B901CD
:10722100A9BCAABDABBEACBF861522E51524205072
:10723100037515DFE51575F004A454FCF5C685F05A
:10724100C722E51724204028E51775F00484A8F02B
:107251000824A8F5C675C70375B901A9BCAABDABB9
:10726100BEACBFA61589BC8ABD8BBE8CBF1248EED1
:0272710022E415
:10727300F516F51579FF12722C75B901E5BCB4FF4B
:10728300040516A9150515E515242050E989157976
:10729300FF75C70375C6A875B90109E5BC04601B72
:1072A30009E5BD04601509E5BE04600F09E5BF04E7
:1072B300600905C6E5C6242050DD09891722751625
:1072C3000075150112722C75B901E5BC20E70205A2
:1072D300160515E515242050EB227900E975F00415
:1072E300A454FCF5C685F0C775B901E5BC20E730A9
:1072F30078D066702B08E5BD66702508E5BE66701C
:107303001F08E5BF66701905C675B90108E5BC66B7
:10731300700E08E5BD66700808E5BE667002D322EC
:1073230009E9242050B6C32212734B127333A80108
:107333007F08E0F608DFFB2212734B127343A801A8
:107343007F08E6F008DFFB2278D0796275A7047521
:107353008307EBC454F0F5822212722C78D0127397
:1073630076E5BCF9C23C20E702D23C127376786220
:1073730012737675B901A6BC08A6BD08A6BE08A6F9
:07738300BF0805C622D2205D
:10738A0012722C78D012739A12739A786212739AC4
:10739A0086BC0886BD0886BE0886BF081248EE0568
:1073AA00C62212628C12D1E6127B2C02D02612D18E
:1073BA00E67F007E09909700126C0C7F0A7E12E528
:1073CA00150412C60D7F1412BDD312188F7F277EA3
:1073DA000875130778D0126C8AE6793E30E702798D
:1073EA002F7E34E912C7697F3D7E01909830126C76
:1073FA003F20311B303003128624C23B12766812BA
:10740A00741ED23B1276681274301276AF807C12E8
:10741A00B44980E6C23B7F447453201702744E7EFF
:10742A000012C7698017D23B7F4F74572017027426
:10743A00457E0012C7697E06E51E12C7567E0CE518
:10744A001D12C7567E12E51C12C7567E17746412A7
:10745A00C7697E1CE51B12C7567E22E51A12C7565B
:10746A007E28742E302602742712C7697E2DE519EC
:10747A0012C7567E33E51812C7567E39302607746E
:10748A002C12C7657E3BE53702C756742D201702BA
:10749A00742B7F707E1512C7691274B37E3A12C5B7
:1074AA00B67E0190985B026C0C7E1BE51C12C756D7
:1074BA007E21E51B12C7567E27E51A12C7567E2D76
:1074CA00E51912C7567E33E51802C75612755412CB
:1074DA00757F1278561273B81278AE20171E1002F2
:0774EA001B1243E512BBE891
:1074F10012753C12189A7F347E2F126C971273F119
:1075010012D02680E212188F203026203128C23B6B
:107511001276681275947866127768D23B12766893
:107521001275A978691277681276AF1276230278FC
:107531000B1286ED80F212B45E80EDE57D75F010E0
:1075410084AAF075F00AA42A547FFA78D7E6548009
:107551002AF6227F277E0879D08700C001D224B97C
:10756100D002C224127935D001A70010230909EEF7
:107571002406FEB9D7E32219EE24FAFE80DB7E341D
:1075810079D7E7A2E792171278E279D7E7A21792A3
:10759100E7F722C224C23B751E007F447E001278A9
:1075A100F2801E1023ED802AD23BC2247F4F7E0041
:1075B1001278FAD2247E06E51E127927F51E1023D1
:1075C100E7D2247E0CE51D127927F51D303BD4103E
:1075D10023E1D2247E12E51C127927F51C1023E148
:1075E1007E1CE51B127927F51B1023E67E22E51A86
:1075F100127927F51A1023E87E2DE519127927F55E
:10760100191023E87E33E518127927F5181023E8BD
:107611007E393026027E3BE537127927F537102374
:10762100E3227F707E151278EAC2247E1BE51C12CC
:0A7631007927F51CD2247E21E51B09
:10763B00127927F51B1023E77E27E51A127927F518
:10764B001A1023E67E2DE519127927F5191023E878
:10765B007E33E518127927F5181023E82278D7E640
:10766B00C2E775F00A847866F537303B0578698593
:10767B00F0371276D830262BE53775F003A40404C7
:10768B0075F00584FBE51975F00AA4251875F0064D
:10769B00A42BFBE435F0FC125E08F537125E08F5FF
:1076AB00188B1922E563FC339217AB625003125E01
:1076BB0079305C0A7AD2125BF47840125D96AE0494
:1076CB00AF037C277D10125CFF8F1C8037E6FD33E8
:1076DB0092171886041886035003125E817A097973
:1076EB002778C0125D938B1EADD3ACD2AB0679EA73
:1076FB007860125D918B1DAF06AED27C177D701238
:10770B005CFF8F1CAF05AE047C037DE8125CFF8F22
:10771B001BAF05AE047C007D64125CFF8F1AED7508
:10772B00F00A84F51985F01822EC339217500312E6
:10773B005E79751D30301786751D2D808178427BE3
:10774B00607CEA800678407B207C4E12B529792735
:10775B007810125D918B1CAF06AED280AB30262A0F
:08776B00E51975F00AA42518C8
:1077730075F00AA42537FBE435F0FC7A05125BE6C5
:107783008C068B077C007D03125CF28E048F031240
:1077930076A2E51E75F00AA4251D75F00AA4251C22
:1077A30075F006A4251BFBE435F0FC7A0A125BE6B0
:1077B300EB251AFBE43CFC7A0A125BF4EB2519FB7C
:1077C300E43CFCE43DFD7A0A125C06EB2518FBE47D
:1077D3003CFCE43DFD301703125E81A60518A604A8
:1077E30018A60378D7E6A2E7923DC2E775F00A84AC
:1077F300FCABF0303B0EAB37EC75F00AA42BA23D8B
:1078030092E7F622AC3780F0127826305C0A7A4091
:10781300125BF478D2125D96301703125E798C6393
:107823008B62221278367A0A125BE6EB2518FBE4A8
:107833003CFC22E51C75F00AA4251B75F00AA4255F
:107843001AFBE435F0FC7A0A125BE6EB2519FBE43C
:107853003CFC2212788812D0B9C202C22312788863
:1078630010000810010510021B80F51031ED1030D7
:107873000D102604D22680E3D230C23180DDD2310E
:04788300C23080D7B8
:10788700227F35909819126C3D90983720300F90D1
:1078970098532031099098282026039098201F7E1E
:1078A70017126C0C02D0267F357E01909355126C0F
:1078B7003F7F347E3A1279D7744E12C76912D026A9
:1078C70012D0B9C2027F347E3AD217751159751298
:1078D7004E802675112E751227801E75113E751262
:1078E7002F801675112B75122D800E75114E75127E
:1078F7005380067511457512571279D7E511301760
:1079070002E51212C76912D02610000810010510EF
:10791700020B80F5D23C1017E3D21780DF0279D231
:107927004430F8127931E8540F22C2218002D22163
:10793700A224922292231279D7E830E709D23C7425
:1079470030302102745FF812C76912D02610003454
:1079570010010510025D80F5D23C102266102367E6
:10796700B43909745F2021DF743080DBB45F04749D
:107977002D80D4B42D04744180CDB45A0474308062
:10798700C60480C3D23C302406102237102338B4F3
:107997004104742D80B1B42D04745F80AAB45F04D0
:1079A700743980A3B43009745A20219B74398097A5
:1079B700148094B47108D223E812C769800DF8C205
:1079C70023800874718001E802794E9079EC800376
:1079D7009079E8C007EF2408FF12C797D00702D0B5
:0979E700260205F8F80205000073
:10CF7D0075A70090CFAF75F02D84C2D5C2D16017C3
:10CF8D00D2D1146007D2D514600DC2D1E5F093FC57
:10CF9D00742D95F093FB22E5F093FB742D95F09392
:10CFAD00FC220009121B242C353E474F5860687037
:10CFBD007880888F969DA4ABB2B8BEC4CACFD4D9A1
:10CFCD00DEE2E6EAEDF0F3F6F8FAFCFDFEFFFFFF18
:10D06B00D23D8002C23DED8BF0A430E70205F0C348
:10D07B00E895F020D50425F025F0FEED8CF0A430DA
:10D08B00E70205F0C3E995F030D10425F025F0FF58
:10D09B00203D0B2487500122EF24CC40012202D1EA
:01D0AB002B59
:10C9E700203A7A7E1C7F5312D12B7F5912D12B1EEE
:10C9F7007F5712D12B7F5512D12B7E2312D12B7F3C
:10CA07005712D12B1E7F5912D12B7F5312D12B1FB7
:10CA17007E2012D12B7F5A12D12B7E1E12D12B7F53
:10CA27005212D12B12096EE5BD20E0143006117F9A
:10CA3700357E1C90CAA7E571700390CAB102C797EB
:10CA4700E5716018E57012CF7D781F79567D091260
:10CA5700D06F303A0312CA7A0DBD16F3227E1C7FBF
:10CA67005390CA9012C797200CD67E1F7F4112BEE3
:10CA77002F80BCC0060E30D5021E1E12D12BD00649
:10CA87001F30D1020F0F02D12B070700386C446CFF
:10CA9700380005052070D8702005057088A88870B3
:10CAA700080710387CFE383838000807102844C6B5
:04CAB70028283800F3
:10BC0D009098657F717E23126C3F12096EE5BC7EA4
:10BC1D003112C72430121AC23C12096EE5BCFB75F5
:10BC2D00F00AA4F904FAC23D12B1C712BE9B303D11
:10BC3D000122DAF712BDB37C00EBF4042E4019ADEE
:10BC4D0003125CF2EFA2D1203C077E237F6502C375
:10BC5D0083AE16AF1702BD54AD01125CF2EF12C4E4
:10BC6D0071203C077E237F6502C3A7AE16AF170276
:10BC7D00BD787F567E0512BDDF7F3D12BDF27F6F11
:10BC8D0012BDF27E1F7F4112BE2F7E0A7F4112BE72
:10BC9D00517E227F5912BE512012012212B1C78549
:10BCAD007A1D855E1C857B1B855F1A7AC0C23D128D
:10BCBD00BE97203D5212BDB37C007D14125CF27410
:10BCCD00562F20D1029F9FFF24CB40028037EF24B7
:10BCDD008850028030EA1475F00384FE12D12BC314
:10BCED00E51B957BFEE51A955F92D55004EEF404A5
:10BCFD00FEEEC313FE24E0400C741F2E30D5029EC1
:10BD0D009EFE12D12BDAA8227F5212BD277F5A1226
:10BD1D00BD2775175375160080287E0012D15B0E56
:10BD2D00BE12F922201201227F157E2B742012C71C
:03BD3D00697F1CFF
:10BD40007E2B12D15B0EBE40F975171575162DD2DC
:10BD50003C02BC26C23D6002D23D92D175F08030DB
:10BD60005C04F5F08001A4A2E792D5E5F075F0320D
:10BD700084F8E5F075F00584C0E0E5F0A2D533C0A5
:10BD8000E0E8601E12C756EE2406FED0E0F8D0E0D0
:10BD900012C756EE2406FE742C12C7690E0EE80276
:10BDA000C7567420303D07742B20D102742D12C762
:10BDB0006980D4C3ED957AFFEC955EFE92D1500375
:10BDC000125E69227F1512BDCB7F327E3E12D12BCF
:10BDD000DEFB227E0912D12B0EBE36F9227E011225
:10BDE000D12B0E0EBE3FF8227E3312D12B0EBE4059
:10BDF000F9227E047D1112D12B0E0E0EDDF81F1FCD
:10BE00007E3590986E305C057E31909872026C3F62
:10BE10007405305C097E32740112C72474067E36C4
:10BE200012C7247E3A740012C7247E3D02C7247DC7
:10BE30000F12D12B0F0F0FDDF8227F737D038004CB
:10BE40007F727D0512D12B0FDDFA227F717D078075
:10BE5000F37D0A12D12B0E0E0F0FDDF722203D07C6
:07BE60001237937003D23D7D
:10BE670022056D12AF68E4F5F7C2B2C2B2ABF7F5BF
:10BE7700F7C2B2C2B2E5F7FA30E411EB251DF51DA2
:10BE8700E4351CF51C0519EA30E3010ED2B2801522
:10BE9700780380027801203D071237937003D23D63
:10BEA70022D8F3056DE56D2409F56D12AF68E4F549
:10BEB700F7C2B2C2B2ADF7F5F7C2B2C2B285F71B8D
:10BEC700F5F7C2B2C2B2E5F7FCD2B2C220543F3096
:10BED700E50244C0CC54C02323F51AE56D24F6F5DA
:02BEE7006D22CA
:10C90E007E017F0990C98C12C7972051097E037F43
:10C91E0000743F02C769E4FEFFC3E54512C16FFD17
:10C92E00940AED403D9464ED4002746312C6077E96
:10C93E00017F09E552240575F02D84AAF075F005E6
:10C94E00A4CA75F00B842A90C9779312CF7DBCB818
:10C95E00027BB87D04EE2DF8EF2DF90D12D06BDDB4
:10C96E00FB227E0312C75680C6000C1622222D39DA
:10C97E00444F4F5A66707C7C87939EA9A900090983
:10C98E000800410000000000888000000000410007
:10C99E000800120982E5BCB4F8339004C3E0602CA1
:10C9AE00FA24F340277F137E0012D12B0F0F12D1E2
:10C9BE002B0E12D15B1F1F12D15B0EDAEC7F147E91
:10C9CE000012D12B0E12D15B0EBE12F5229005CCA9
:09C9DE00E0C3941240F60480C786
:10C16F00305D0A75F08AA42480E5F03400227F0048
:10C17F002074147E110F90C20D12C7977F0A7E0A8A
:10C18F00E52E540702C61E7E0BE571B4FF2DE55157
:10C19F0024025003755100E55112C16F75F005A4CB
:10C1AF00ACF0FB125BBC7E0D781CE66004E612C798
:10C1BF004FEE2405FE18B818F4800612C16F12C690
:10C1CF000D7F0C7E11E571602F0EE57064B4602851
:10C1DF0064B475F03284C0F012C74FCE2405CED0B0
:10C1EF00E075F00584C0F012C74FCE2405CED0E025
:10C1FF0023302D010402C74F907D1B026C0C070FDB
:10C20F00FFFF9EE7AD6B9C6BAD6B9D67FFFF75549A
:10C21F008030745F78BD79BBE6FC27FB1819E6FD0B
:10C22F0037F9EBF87B00125D988B547F087E11A8CD
:10C23F000690C28312C79730101120730E7F0A7EAB
:10C24F001712D15B0E0E12D15B7F08E5542483E5E4
:10C25F0054500224FA75F01984FB90C28B9328FE78
:10C26F00EB90C29593FD12D12B0F0F12D12B1F1FE5
:10C27F000EDDF322030F0100FFFE0380000000001C
:10C28F0007070D0C0B0A0504030201010203040545
:10C29F00306701227F357E00746F12C769E57E60BB
:0DC2AF00F212C16F75F06484F87E06E5F0B0
:10C2BC0012C66CE860E07E0002C756202C0122906A
:10C2CC00C2D102C797050EFFF0E01CF004F81CFF6A
:10C2DC00F0301201227F6E7E0090911A12C7977F68
:10C2EC001512BDCB7F1F12BDCB7F2912BDCB7F1783
:10C2FC007E06E53F30E00B909882305C0390989678
:10C30C0080132074077E0190913A800990987730C1
:10C31C005D0390988C126C0C307306E54E60021520
:10C32C004E205718E54EB40113120991C3E55C95E4
:10C33C0060F5BCE55D9561F5BD1248EE7F217E018F
:10C34C00E53F30E02130570590920F8016E54E7096
:10C35C000590921B800D909146126C0C7E30E54E30
:07C36C0002C672126C0C22E4
:10C4D900125B8E7F207E05751900781DC2D5E63066
:10C4E900D51712C74FEE2405FE18B818F17E1F7430
:10C4F90063305C02746502C7697005B8191880E277
:10C50900D2D5CE24FACE746B301702742D12C769B6
:10C51900EE2406FE80C8742012C76580C8781C8086
:10C529000D7F007E23AC5EAB7A125B8E781DC2D57F
:10C53900E630D50C12C756EE2406FE18B818F122BB
:10C549007005B8191680EDD2D53017E4CE24FACE8D
:10C55900742D12C769EE2406FE80D5742012C769AE
:10C5690080D5125B8E781DC2D5E630D51612C72448
:10C57900EE2404FE18B818F10E745E305C027427BC
:10C5890002C7337005B8191680E3D2D53017DACE51
:10C5990024FCCE742D12C737EE2404FE80CB742000
:10C5A90012C73780CBC23D12C5C10F0F0E0E74637F
:10C5B900305C02746502C769125B8E781DC2D5E6CC
:10C5C90030D50C12C786EE2408FE18B818F122706F
:10C5D90005B8191680EDD2D5301716740BCE24F88C
:10C5E900CE12C786EE2408FE80D5740C12C7868049
:08C5F900D5303DCB740A80E54A
:10CABB007F797E24E55F30E70122AC5F1CAB7B12F4
:10CACB005BBCE51B700E742012C769EE2405FE12C9
:10CADB00CB09800C12CB09E51B12C74FEE2405FEC8
:10CAEB00E51A12C74FEE2405FE742C12C7690E0E01
:10CAFB00E51912C74FEE2405FE745E02C769742D4B
:10CB0B00201702742B12C769EE2406FE22E55F3054
:10CB1B00E70122AC5F1CAB7B125BBCE51B700E7498
:10CB2B002012C737EE2404FE12CB62800C12CB62AC
:10CB3B00E51B12C724EE2404FEE51A12C724EE24CB
:10CB4B0004FE742C12C7370E0EE51912C724EE24FF
:10CB5B0004FE742A02C737742D201702742B12C7D8
:06CB6B0037EE2404FE2257
:10C373007F097E2530040512C46D8028A275E579F6
:10C38300C23D6002D23D92D175F080305C04F5F07D
:10C393008001A4A2E792D5E5F075F03284F8E5F0C8
:10C3A30075F00584C0E0E5F0A2D533C0E0E8602A6B
:10C3B30012C786EE2408FED0E0F8D0E012C786EE5E
:10C3C3002408FE0F0FE52B5403701F746012C76916
:10C3D3001F1FEE2404FEE802C786740C303D06746A
:10C3E3000A20D1010412C78680C9205904742E8003
:10C3F300DC205804746180D5746280D13004051246
:10C40300C46D8028A275E579C23D6002D23D92D108
:10C4130075F080305C04F5F08001A4A2E792D5E5C5
:10C42300F075F03284F8E5F075F00584C0E0E5F0CE
:10C43300A2D533C0E07F3E7E1CE8602012C7E7D060
:10C44300E0F8D0E07F3E7E2812C7E77F447E327457
:10C453002E12C7697F3E7E37E802C7E7303DE0749E
:10C463000A20D1010412C7E780D59005CAE075F010
:10C473000A84F8E4C5F0C2D522301105E54AB402B6
:10C4830050C39006E9E0957AFB9006E8E0955EFCE0
:06C493005003125E79EC7B
:10C49900C31360047B63800FEB13FB249C40F524DA
:10C4A9004F4004C20480079005CAEBF0D2049006FD
:10C4B900E6E09006E8F09006E7E09006E9F0E55E30
:10C4C9009006E6F0E57A9006E7F02212C4B780DE1E
:10BEE900E54424F64001227800E552206607C3950F
:10BEF90070500224B40475F00384F9E928FE24C4BF
:10BF09005001FE12BF2B12BF371E12D12BC3E99865
:10BF1900FE5003243CFE12BF2B1E12D12B08B81F62
:10BF2900DA22EE2420FE24C250032402FE22E82451
:10BF3900F1E8C2D55006D2D5E8F4241F23FF90BFFB
:10BF4900B993CF0493FAE545F5F0A4ACF0FB125C84
:10BF59001DE544F5F0A49BFBE5F09CFCEB2420FBDC
:10BF6900EC3400FC12BF9AFAE5458FF0A430E702E1
:10BF790005F0E5F020D502F4042A75F0052019032F
:10BF890075F00384FF24DF50027F20C374329FFFC2
:10BF990022EC24F0500BEB2460EC340090C00993A0
:10BFA90022EB33FBEC33FCEB33EC3390BFD9932218
:10BFB900FF00FF03FA0BF318EA2ADE40CF58BE73DD
:10BFC900AB8D96A880C068D64FE835F51BFD00FFFC
:10BFD90000080B0E101214151718191B1C1D1E1F13
:10BFE90020212223242526262728292A2A2B2C2DDD
:10BFF9002D2E2F2F30313132333334343536363715
:10C00900373839393A3A3B3B3C3C3D3D3E3E3F3F70
:10C019004042444648494B4D4E5052535556585943
:10C029005B5C5D5F60616364656668696A6B6D6EC0
:10C039006F7071727374767778797A7B7C7D7E7F85
:10C04900808182838485868788898A8B8B8C8D8E73
:10C059008F9091929394949596979899999A9B9C7D
:10C069009D9E9E9FA0A1A2A2A3A4A5A6A6A7A8A99A
:10C07900A9AAABACACADAEAFAFB0B1B1B2B3B4B4C9
:10C08900B5B6B6B7B8B9B9BABBBBBCBDBDBEBFBF03
:10C09900C0C1C1C2C3C3C4C5C5C6C7C7C8C8C9CA48
:10C0A900CACBCCCCCDCECECFCFD0D1D1D2D2D3D496
:10C0B900D4D5D5D6D7D7D8D8D9DADADBDBDCDDDDEC
:10C0C900DEDEDFDFE0E1E1E2E2E3E3E4E5E5E6E647
:10C0D900E7E7E8E8E9EAEAEBEBECECEDEDEEEEEFA9
:10C0E900EFF0F1F1F2F2F3F3F4F4F5F5F6F6F7F710
:10C0F900F8F8F9F9FAFAFBFBFCFCFDFDFEFEFFFF7F
:10C10900E54524FD400122E552206607C39570509C
:10C119000224B40475F00384241FFE24C2500324AE
:01C129000213
:10C12A00FE12C164EEFD241EFE24C250032402FE48
:10C13A0012C164E544240275F00520190375F00361
:10C14A0084F4042432FF24EE500F12C159AE051EA6
:10C15A001E7C0512D12B0EDCFA227F1512D12B0F71
:05C16A000FBF2DF822BB
:10C826007E00206615E5700475F0B484E5F075F0B9
:10C836000384FE6004C3743C9EFE745312C8517494
:10C846005712C851744E12C85174457F2F12C737FC
:10C85600BE00077E3C12C7377E00EE240875F03C0A
:10C8660084AEF00F0F0F12D12B0E12D12B0F12D157
:10C876002B1E12D12BEE240775F03C84AEF022302D
:10C88600745C301259E54AB4040122B4060122E56B
:10C896007112BF838F057C037E1E30662AE5700405
:10C8A60075F00384241EFE24C6501C24FB50042469
:10C8B600038013C00612C8CDD0E024C67C016006F2
:10C8C6000C1460020C14FE12C8D90EEE24C14002EC
:10C8D600DCF5228D0712D12B0FEF24CE50F722E57F
:10C8E60053206607C39570500224B40475F0038480
:10C8F600241FFE24C250032402FE12C9040E7F2305
:08C9060012D12B0FBF2DF92205
:10CFDD00AF177E00E53C12C6017E0C742E12C76998
:10CFED007E12E53B12C6017E1E742E12C7697E2489
:10CFFD00E53A02C6017E0E78ADE612C66C7E187457
:10D00D002C12C7697E1B18E612C66C7E25742C1275
:09D01D00C7697E2818E602C66C02
:10D0EC007F797E16743B12C7657E18E53F12C66CBD
:10D0FC007F797E0078AEE612C66C7E0A743B12C74E
:10D10C00657E0CE53E02C66C7F797E00E54012C65A
:0FD11C006C7E0A743B12C7657E0CE54102C66C3F
:10CCCE00787512CD1E7453201702744E207406E52B
:10CCDE002E54074430AF1712CD487E3BE57DC45429
:10CCEE000F12C7562074077E07742012C769787812
:10CCFE0012CD1EE5172409FF745720170274452024
:10CD0E007402742012CD487E3BE57D540F02C75647
:10CD1E00E6FD339217188604188603301703125E49
:10CD2E008179177870125D918B13AF06AED27C00AD
:10CD3E007D64125CFF8F148D15227E0012C7697EF2
:10CD4E0007E51312C61E7E19746412C7697E20E5AC
:10CD5E001412C6017E2B742E2073030E742C12C770
:08CD6E00697E2FE51502C601E4
:10CE8F00E54A602E7A2420E00E7A26141460087A80
:10CE9F0028141460027A297F717E00EA12C7692074
:10CEAF005505205406800B745B8002745C7E001263
:10CEBF00C76920110778A9B60007802F30262CC22A
:10CECF00269099BE7F68126BFA7F66A85AE54AB41E
:10CEDF00060108E875F06484740AC5F084C0F01286
:10CEEF00C786EE2409FED0E012C78620080FE5376B
:0ECEFF00640260097F367E2E744112C737220E
:10CB710020144F740512D1D2EF33EE33F9EF0303D2
:10CB8100541FF5F090CBC4E993A4C5F013C5F0137D
:10CB9100C5F013C5F013C5F0135403FCE5F013FB06
:10CBA100E9242093C9244093C39BC4540FFBE99CFF
:10CBB100C4FC540FF9EC54F02B2446F57BE934F610
:10CBC100F55F22FFFFFFFFFFE6C5AD9C8F857D77F7
:10CBD100726E6C6A696A6A6C6F747A828D9DB4D95F
:10CBE100FFFFFFFAE9DCD3CEC9C6C3C0BEBBB9B7EC
:10CBF100B5B4B2B0AFADABAAA8A6A4A2A09E9C99B1
:10CC010096918C00381CE735D137246F00C5B3C12C
:10CC1100E61F66B60E68C21867AADBF4EDB9467561
:03CC210010A2005E
:10D1B200D2A27408D2A1D2A300C2A3C2A1D2A30058
:10D1C200C2A3D5E0EF7405D2A300C2A3D5E0F82232
:10D18B00C2A3D2A2D2A1D2A300C2A375F00833923C
:10D19B00A1D2A300C2A3D5F0F5C2A175F003D2A30F
:07D1AB0000C2A3D5F0F82239
:10B8320012D18BD2A300C2A3C2A175F008E4D2A395
:10B8420000C2A3A2A233D5F0F5FE75F008E4D2A39C
:10B8520000C2A3A2A233D5F0F5FFD2A300C2A32255
:10B86200E478806608B88BFB70012274D512B83276
:10B872007881C3EE13FEEF13F692D118EE2460F630
:10B8820074D612B8327888EF33CE33CE33CE33CE7D
:10B8920033A2D192E25407FCEEFB7A08125BE6EC8B
:10B8A200244FF608EBF674D912B832EF543F78827F
:10B8B200F67886EF33CE33CE33CE33CE335403F61F
:10B8C20008EEF618161608E6C4FF54F0F618E6C499
:10B8D200CF540F2FF674DA12B832EF232354FC78C8
:10B8E20083F67884EEF608EF54C0F67880E46608B2
:10B8F200B88AFBF62212B83A7889C3EF96FF18EE9F
:08B9020096FEA2E79216501018
:10B90A00125E69740FF8F9125C33EF2CFFEE3DFEFC
:10B91A00788BEEF608EFF622E6182016072CF7E6E3
:10B92A003D19F722C39CF7E69D80F66A405E805671
:10B93A00E050F04B0044803DC0384031D02BA02568
:10B94A00601F2018D014000F000AA00144015801FA
:10B95A00680178018801A001B401D001EC0210024B
:10B96A0038026802A002DA030C034D78BE802085F3
:10B97A008E8A9D8F4D95BA9A97A0BEA631AC53B2C6
:10B98A002AB801BD6AC1EDC4D1C78812B83A788D08
:10B99A00EEF608EFF67887798C125C337883799023
:10B9AA0012B9227885798C125C337881799212B92E
:10B9BA0022788DE624E4FE08E63392D13392D554F8
:10B9CA00FCFFEEA2D133A2D533FE780F7992125C36
:10B9DA003378947990C3EC97F61819ED97F6799421
:10B9EA0090B9357F1F7D11EF93C3971F19EF939776
:10B9FA001F091DED600240EF0F90B955798DEF9345
:10BA0A00F7090FEF93F7788E7994125C3390B97532
:10BA1A00EF93C39BFB1FEF939C2420FC7897E62BA4
:10BA2A00F618E63CF618E436F6740612D1D2D23786
:09BA3A00EE24F74006240250023C
:10BA4300C237EEFCEFFD740712D1D2C3ED9FFFECBA
:10BA53009EFE78B7E6FD337C0050011CEF2DFFEE10
:10BA63003CFE78D8E6C4540F2FFFE43EFE789CEFEB
:10BA730026F618EE36F62220141220370F789DE6AC
:10BA8300B4050912BB3212BB6712BBB02220145E8D
:10BA93007897799A12BBCB125DF1C3EE9420FE9294
:10BAA300455003125E697C007D05125CFF3045033F
:10BAB300125E69E531B40C3612CCB4120987E5BCC9
:10BAC3002FF560E5BD3EF56120E71124F8500DFA2E
:10BAD300C3E5609AF560E5619400F561120991E5AB
:10BAE300BC2560F57AE5BD3561F55E12CCC178976A
:10BAF300799AC3E697FB1819E697FC7A02125BE67C
:10BB030030370B7A02125BE6ECFEEBFF800312BBCD
:10BB13003212BB6720140312BBB078957998E6F70D
:10BB230076000809E6F776000809E6F77600227939
:0CBB33009CE77700FB19E77700FC789D89
:10BB3F00E6B40506EB33FBEC33FCECA2E792D550F1
:10BB4F0003125E797A32125BF4ECFBEDFC30D50315
:10BB5F00125E79ECFEEBFF22EE2408FE7404203710
:10BB6F00167406307511789DE6B40504740C8007C1
:10BB7F00F42406C323540FFD7C00125BD2789FE69A
:10BB8F00FC08E6FBC374109DFA125BF4EFF8EEF9B4
:10BB9F00125DF1E878A02FF6FF18EE39F62480FE3B
:10BBAF002292754003125E69EF33EE33F579C27658
:10BBBF00307508E57924F15002D27622E627FB187A
:10BBCF0019E637FC1819E637FD2212B16E7F087897
:10BBDF0071793A12BBF40245B0855E63857A62785B
:10BBEF007379647F06E6F70809DFFA2278647973C0
:0EBBFF0080F1787379AF80EB78AF797380E5D1
:105B6C00E4FEFFFC7D0A791DE7540F2FFFE43EFE97
:105B7C00B91902800619125BD280ED301703125E40
:105B8C006922305C2BEC3392175003125E79EC24B3
:105B9C00D950047C277B007AD2125BF4EB33CC33E4
:105BAC00CD33CC33ED33FBEC33FC301703125E7981
:105BBC00EC3392175003125E797919125E08F709CB
:105BCC00B91DF8A70322EFF88DF0A4FFEDC5F0CEB8
:105BDC00A42EFEEC88F0A42EFE22EB8AF0A4FBE5AA
:105BEC00F0CC8AF0A42CFC22EB8AF0A4FBE5F0CCE0
:105BFC008AF0A42CFCE435F0FD22EB8AF0A4FBE542
:105C0C00F0CC8AF0A42CFCE435F0CD8AF0A42DFD68
:105C1C0022EB8AF0A430E70205F0E5F0CC8AF0A480
:105C2C002CFBE435F0FC2286F0E7FDA4FAABF0196E
:065C3C00E786F0A42BFB3B
:105C4200E435F0FC18E68DF0A42BFBEC35F0FCE417
:105C520033FDE687F0A42CFCED35F0FD22EB89F054
:105C6200A4CBAEF08AF0A42EFEE5F03400FDEC8960
:105C7200F0A42EFEE5F03DFDE433CC8AF0A42DFD28
:105C8200E5F03CCEFC22EB89F0A4CBAFF08AF0A485
:105C92002FFFE5F03400FEEC89F0A42FFFE5F03E83
:105CA200FEE433CC8AF0A42EFEE5F03CFCED89F054
:105CB200A42EFEE5F03CFCE433CD8AF0A42CFCE5F6
:105CC200F03D8E058C068F04FF22C2D5EC30E7052D
:105CD200B2D5125E71EE30E70DB2D5125E69125C7A
:105CE200FF125E718003125CFF30D503125E6922DF
:105CF200C3EC13C0E0ED132FFFD0E03EFEBC000B5F
:105D0200BE0029EF8DF084FFADF022E4CCF975F0EE
:045D120008EF2FFF68
:105D1600EE33FEEC33FCEE9DEC994005FCEE9DFE69
:105D26000FD5F0E9E4CEFD22EDF9F5F0EE8420D2B0
:105D36001CFEADF075F008EF2FFFED33FD4007991F
:105D46005006D5F0F222C399FD0FD5F0EA22EC33C6
:105D5600EE3400FEEF3400FF7D007A00790078090A
:105D6600C3ED9AFDEE9BFEEF9CFFB392D54009ED85
:105D76002AFDEE3BFEEF3CFFA2D5E933F9ED33FDFC
:105D8600EE33FEEF33FFD8D92279007A00C38015AF
:105D960079007A00C3EA13FFE913FEE8132BFBEE42
:105DA6003CFCEF3DFDE4F5D2F5D333FE7F19C3EE9F
:105DB60098FEE5D299F5D2E5D39AF5D3B392D540BC
:105DC6000DEE28FEE5D239F5D2E5D33AF5D3A2D5C4
:025DD600EB33AD
:105DD800FBEC33FCED33FDDF0122EE33FEE5D2337D
:105DE800F5D2E5D333F5D380C3EDC454F0FEECC44B
:105DF800FF540F2EFEEF54F0FFEBC4540F2FFF2279
:105E0800EC75F00A84FCEB54F025F0C475F00A84B4
:105E1800C4CBC454F025F0C475F00A842BFBE5F01C
:105E280022AC10AB11125E08A904AD03FA7C197BF1
:105E380099125BE6AE04AF03EA75F006A4F8AC125B
:105E4800AB13125E082875F00A8485F014F8EF2B5E
:105E5800FFEE3CFEEF28FFE43EFEE43DFDE439FCA6
:105E680022C3E49FFFE49EFE22E4C39DFDE49CFC64
:105E780022C3E49BFBE49CFC22C3E49BFBE49CFC64
:105E8800E49DFD2275D4107B807A0079807800EA41
:0A5E9800F5F0A4FCADF0EBF5F0A46A
:105EA200FEAFF0EB8AF0A4C333C5F033C5F092D550
:105EB2002DFDC5F03EFEE430D501043FFFB5150DC2
:105EC200EEB51409EDB51305ECB51201224006EA50
:105ED20098FAEB99FBD5D40ABB0001220ABA000159
:105EE2000B22C3E913F9E813F8EA28FAEB39FB802D
:105EF200A478087B807D807C00EDF5F0A4FAE5F0C3
:105F02008EF0B5F007EA8FF0B5F001224003ED9B69
:105F1200FDD827BDFF0122EDF5F0A4F9A8F0ED04AC
:105F2200F5F0A4C399FAE5F09813CA1329F9E83AEF
:105F3200F8C3E99FE89E50010D22C3EB13FBED2B42
:105F4200FD80B67473F8F9E627FB0809E637FC080A
:105F520009E637FD30E703125E81EB33FBEC33FCDD
:0B5F6200ED3323FD242083F8ED241C08
:105F6D0083FFED241883FAED241483F9EF99F9E8F2
:105F7D009AFA125C5FEF9DFFE89EFE22FFFFFFB6CF
:105F8D00FED7FD63FB5DF8C4F59BF1E3ED9EE8CF15
:105F9D00E379DD9ED743D06BC919C153B91CB079D4
:105FAD00A7709E06943F8A237FB674FF6A045ECB6A
:105FBD00535B47BB3BF1300423FB17DE0BB2C21D15
:105FCD00C232532CF8C3E5679576FBE5689577FCEF
:105FDD00E5699578FD30E705D261125E8124F050B8
:105FED000312609FAA06A907125C88EC2480E43D89
:105FFD00FBF9F51AE43EFCFAF519E43F6002D232E2
:10600D00125C5F8B128C138D148E15C3E564957322
:10601D00FBE5659574FCE5669575FD30E705D26287
:10602D00125E81EBF9F51FECFAF51DED6002D2322F
:10603D0030320122125C5FEB2512F512EC3513F5AF
:10604D0013ED3514F514EE3515F51540E1025E8CA2
:10605D00125FCB20323BEB242E40D3EA2401CB340C
:10606D0000FC7A07793D125C5FC010C0118E108D57
:10607D00118C128B13E4FCFD7E077FD012A8E885EE
:10608D001203851302D011D010BB0005BA0002D245
:10609D001D22B261C374809BFB74F59CFC74209D22
:0160AD00FDF5
:1060AE0022204D7D20487A303F777F747E0112BDCD
:1060BE00DF7E1F12BE4B75A7009004EDE0A2E792A3
:1060CE00171392E7FC1582E013FB301703125E796B
:1060DE00BC004EEB604B20E74820E64510E5132050
:1060EE001707C3741F9BFE80027E1F12BE400EDB7D
:1060FE00FA22FB2017097E00C374209BFB8008EB5D
:10610E00241FFE74209BFB12BE3A0EDBFA2275A7EB
:10611E0000758307E559C4440FF582E0A2E7925259
:10612E00222212BC0112611CC2E775F00A84FEAF76
:10613E00F075A7045382F1786412619DAE077867FB
:10614E0012619D75A700E57DC4540FFEE57D540FC9
:10615E00FF7873126191AE07787612619174AF1267
:10616E005F4712605D120982E5BD75F00AA4F9EA77
:10617E00999004ECF0A3EB95F0F0A2E7923DD23F9C
:10618E0002BC07860308860408860518188006E0F8
:10619E00FBE0FCE0FD7A0A125C0620E70CEB2EF623
:0E61AE0008E43CF608E43DF622C3EB9EF6083A
:1061BC00EC9400F608ED9400F622C2338006204DD4
:1061CC00F92048F6C23F302A0F78A87600223038E2
:1061DC00FCC23878C5864622E54824F640EFE558DF
:1061EC000460EA75A700758307E559C42408F58295
:1061FC00E070DB0582E0FFE54A64046015E54A6463
:10620C0006600F801DEF24BE5029C23878C5864623
:10621C00802175390AEF20E70975390520E60375E9
:10622C0039022038E0EF24C34009D23878C5A6469D
:10623C00754600120982E5BD240DC39F40251261ED
:10624C0030303D1F753901204006D24078A87623A6
:10625C0020522CE55965586026204D23204820D229
:10626C0033801C303319204D1220480F1285C10584
:10627C0059C3E55895595003855859C233C2402229
:10628C00E558B4FF012285581175A704758307E5FD
:10629C004824F65002805C201259202905202A023D
:1062AC00805112BC01E4F516F51775100012631835
:1062BC00E510700312BBFB126331302910E51B256E
:1062CC0017F517F51BE51C3516F516F51C12633E74
:1062DC0012BBFB0510C3E511951050D175A7000238
:1062EC00BC07E55AF51124F6500375110A75A7047D
:0362FC00758306A1
:1062FF0075100012631812633112633E0510C3E567
:10630F0011951050EE75A70022E510C4F582E0E05C
:10631F00F564E0F565E0F566E0F567E0F568E0F552
:10632F00692275A70112668C1239FA75A70422E942
:10633F00F0E51CF0E51BF022E510C454F0F582E007
:10634F00F512E5822406F582E0F511E0F51CE0F583
:10635F001B22202845E558B4FF012275A704758339
:10636F0007E559F5103033066558600205101263C2
:10637F0047E0F513E07F797E3D12C737E5137E398D
:10638F0012C737E5127E3512C73730480B7F7F7E35
:10639F003512D12B0EBE40F9802C2012012275A789
:1063AF0004758306855B10126347E512700B7E3A06
:1063BF007F79745D12C769800D75F06484E5F07E96
:1063CF00397F7A12C6B9E537B40205128445804584
:1063DF00B403028040E51C7006E51B24FB5036E534
:1063EF0011F964B4602F20062CE537600D200C0ADC
:1063FF00C3E99570F9500324B4F9E912CF7D781DE4
:10640F0079547D1D90CA99E53F20E00390CAA012F0
:10641F00D06F12C79775177975161912647075A713
:06642F00009006E3E511F8
:10643500F0A3120982E5BC75F01970040475F01417
:10644500A4951BFBE5F0951CFC92245003125E7984
:10645500ECF0A3EBF0C24FC263EC700EEB24E64008
:1064650002D24FEB24C84002D26322E51C24ED4042
:106475002BAE1CAF1B1266567C007D32125CFFC032
:1064850005EFAF17AE1612C672CE2405CE742C12C8
:10649500C7690E0ED0E02312C66C801B12664D1222
:1064A50064CACE2405CE742C12C769CE2402CEE868
:1064B50075F0058412C74FCE2404CE7422305D02D8
:1064C500746602C769EE243D50047EC37F4B7C0190
:1064D5007DF4125CFFC004C005EF6007AF17AE1670
:1064E50012C672D007D0067C007D32125CFFA8056B
:1064F500EFAF17AE16CE240ACE02C74F12664DEE89
:106505002450305D03EE24A150047EC37F4B7C01F3
:106515007DF4125CFFC004C005EF6007AF177E2F46
:1065250012C6BFD007D0067C007D32125CFFC005C5
:10653500EFAF177E3712C7247E3B742C12C7377E08
:106545003DD0E075F0058402C7243048032074016E
:0265550022E43E
:10655700FCF5A79006E3E0F9A3E0FE24FE40EFA3D5
:10656700E0FF7D78E537600B304FE3200C2F126694
:1065770043802A12096EE5BD20E00F204F07E5464C
:1065870070083063C9D206126643204F107D3CE580
:1065970046600A7D141460057D0A1470B1891112D2
:1065A7005BD27D6F125CF2BE00A4EF24E2409FAD88
:1065B70007E51112CF7D202404B2D5B2D1781F7917
:1065C7005612D06FA806A907E511242D75F0B484DB
:1065D700E5F012CF7D7407304F02740EFDFA12D02A
:1065E7006FB2D5B2D112D06FB2D5B2D1DDF0AD0254
:1065F70012D06F850616850717B2D5B2D112D06FA4
:1066070085061E85071F7A03304F027A06E5112497
:106617001675F0B484E5F012CF7DA816A917AD0260
:1066270012D06FDDFBE51124EA400224B412CF7DBE
:10663700A81EA91FAD0212D06FDDFB22C3E995701A
:10664700500224B4F922E51B2402FFE4351CFE3076
:106657005D1ABEC305BF4D028012AC06AB077A1B9D
:10666700125BF47832125D96AE04AF032278737929
:1066770064125F4912605D751CC3751B4B203204A1
:0E6687008B1C8A1B2212667430320122AC1961
:10669500AE1AA91DAF1FB90005BC00028010C3E9E1
:1066A50013F9EF13FFC3EC13FCEE13FE80E8BF29CB
:1066B500005006BE2900500122C3EF13FFC3EE139D
:1066C500FE80EB3E7FE3E3E3E3E3E3E3E3E3E37F42
:1066D5003E0C1C3C7C7C1C1C1C1C1C1C1C7F7F3E1B
:1066E5007FE3E3E3070E1C3870E0E3FFFF3E7FE343
:1066F500E3030F0E0F03E3E3E37F3E070F1F3F772F
:10670500E7E7FFFF0707070707FFFFE0E0E0FEFFFA
:10671500030303E3E37F3E1E3F73E0E0E0FEFFE398
:10672500E3E3E37F3EFFFFE3E30303070E1C383893
:106735003838383E7FE3E3E37F3E7FE3E3E3E37FFF
:106745003E3E7FE3E3E3E37F3F030303E77E3C0055
:106755000000181818FFFF181818000000000000A6
:10676500000000FFFF0000000000003FF0000038BF
:106775001C38F00180C1F020F0FC0038F03FE0004B
:106785000000007CC6C6C6C6C6C6C6C67C18387814
:106795001818181818187E7CC6C60C183060C0C6A4
:1067A500FE7CC6C6061C0606C6C67C0C1C3C6CCC0C
:1067B500FE0C0C0C0CFEC0C0C0FC0606C6C67C3C1C
:1067C50066C0C0C0FCC6C6C67CFEC6C6060C183070
:1067D5003030307CC6C6C67CC6C6C6C67C7CC6C63E
:1067E500C67E060606CC78000018187E7E181800AE
:1067F50000000000007E7E00000000000000000098
:106805000000000000000000000000000000008003
:1068150080A0C0A000304020C08080C0A0A00000A3
:1068250060A0600000A040A05098D090882050A89B
:1068350050888850A8502060806000000040E040EB
:106845000000000000800000E000000000000040A3
:10685500002040800040A0A0A04040C04040E0C0D3
:106865002020C0E0E0204020E02060A0E020E0C043
:106875002020C06080E0A0E0E020404040E0A0E0B3
:10688500A0E0E0A0E020C0004000400000800080C3
:10689500002060E0602000E000E00080C0E0C080F3
:1068A500E0E0E0E0E0000000000040A0E0A0A0C0C3
:1068B500A0C0A0C040A080A040C0A0A0A0C0E08013
:1068C500C080E0E080C080806080A0A060A0A0E0E3
:1068D500A0A0E0404040E0202020A040A0A0C0A013
:1068E500A080808080E0A0E0A0A0A0A0E0E0E0A0E3
:1068F50040A0A0A040C0A0C0808040A0A0C060C0B3
:10690500A0C0A0A060804020C0E040404040A0A0C2
:10691500A0A060A0A0A0A040A0A0A0E0A0A0A04032
:10692500A0A0A0A0404040E0204080E02020A8702A
:10693500202070A8202008F030D0100000F0A8A872
:10694500000000E000000090204870889898400002
:10695500E0E0E000A0E0E0E0406030103060404062
:10696500E040406090909090906020602020202032
:1069750070609010204080F06090102010906010A2
:10698500305090F01010F080E01010906060908012
:10699500E0909060F0102020404040609090609022
:1069A500906060909070109060C0E0F0F8F0E0C0EA
:1069B5000000000000000000000000000000506022
:1069C5005000707050000078807008F000F88888DA
:1069D50088F800C0C8102040981800C0B098B0C012
:1069E50000602040000000000090D8FCD890000016
:1069F500246CFC6C24000020A870A8200000202036
:0D6A0500F8202000000000000000800000CC
:106A120000F000000000000000006060000810208C
:106A2200408000708888888888702060202020201C
:106A320070708808102040F8F81020100888701034
:106A4200305090F81010F880F008088870304080BC
:106A5200F0888870F808102040404070888870885C
:106A6200887070888878081060006060006060003C
:106A720000008000008000002040F840200000005C
:106A8200F800F80000002010F810200070880810AC
:106A92002000200000000000000070888888F8882C
:106AA20088F08888F08888F070888080808870E01C
:106AB2009088888890E0F88080F08080F8F8808064
:106AC200F0808080708880B8888878888888F88884
:106AD20088887020202020207038101010109060BC
:106AE2008890A0C0A09088808080808080F888D81C
:106AF200A8A88888888888C8A8988888708888887C
:106B0200888870F08888F080808070888888A89053
:106B120068F08888F0A0908870888070088870F883
:106B2200202020202020888888888888708888886B
:106B320088885020888888A8A8A850888850205023
:106B4200888888888850202020F80810204080F803
:106B520000CCAC9CACCC0000CCD4E4D4CC00047807
:106B62001828C800FC40A04018202018000000008F
:106B72000000F800000000A040A0000000600060DB
:106B820060006000600060600000F0A8A8A8A82073
:106B92005020000000005090B890D0908860505073
:106BA20000707050805048FC485080304C5C6060EF
:106BB200603C00E0F0080808F88044485C484480E3
:106BC200008820208870000080C0A090F800304823
:106BD200B4B44830003048B4B44830FC0098D020F7
:106BE20058C8008080F088888888F8E8D880D8E87B
:086BF200F8404050F85040400B
:0300000002005E9D
:03000B0002A978CF
:0C000E00206E06859950D26E32D26F32FF
:0E00230010990AC298206DE385994FD26D3274
:10003800E4F537F534F52F12D0E2C229C22AC26896
:09004800C227C214C2150227BB35
:03005B0002258BF0
:10A96B008530F0C5F065308530F060F722C0D0C07F
:10A97B00E0C0F0C0A775A700C083C08275D0087572
:10A98B008A00300503758A7A758CEA0532E53270D8
:10A99B000215320530E530640A6026201520E531BA
:10A9AB00B40C0BE530B4010612ADC312CB71E5311B
:10A9BB00B4180BE530B4060612ADC312CB7102AB63
:10A9CB0083C2AFD2C075C07AD2AFF5300531E53155
:10A9DB0064197047F53120152AC22C7D0A740412B4
:10A9EB00D1D2EF33EE339005CCF0EE24F5401424A6
:10A9FB0002400E24014008202005DDE102258BD208
:10AA0B0025D22CE5A6600215A678B5E6600116786E
:10AA1B00B6E660011678D8E6600116302E09E536E9
:10AA2B007005C22E12ACF5E5367004C24B800215D0
:10AA3B003678A9E660011678A8E66001160535E5BB
:10AA4B003570021535E590307B0B30E008D278C2BB
:10AA5B007BC200801A307C0B30E108D279C27CC2F9
:10AA6B0001800C307D0930E206D27AC27DC202E54C
:10AA7B009044F8F47003753500E533600515330227
:10AA8B00AB28E590F45407700302AB28A2E09200C8
:0BAA9B00A2E19201A2E292023010033F
:10AAA60020144275330820001B20100C2011098049
:10AAB60013E59030E10E8006E53724FC40F3E543CC
:10AAC600541FF53320100375A6FF78A8E6705320AF
:10AAD6002E50301004E536704920100C201109E57F
:10AAE6003524F55003753304D21BD2A5D2A612AC79
:10AAF600F575B44075B2400534202726206823201A
:10AB06002920202A1DA21072115017E52054076033
:10AB160011E5342438400B200026200119D27D751A
:10AB260034C8201558E531702412D1B274E812D118
:10AB36008B802A02AC42E53724FC40E6D27C80DFDB
:10AB46003011DFE53724FC40D9D27B80D275F00383
:10AB560084E5F070DE12B8F774E812D18BE531B4F3
:10AB6600060512BA7A8016B40C0512BA90800EB495
:10AB7600120512BA7A8006B4180312BA90E590301C
:10AB8600E10530E202800620100D20110A78A8E6C1
:10AB9600705120103C80612027F32068F02029EDB9
:10ABA600202AEAE534243040E4240750E0600B20F4
:10ABB6005E088590F020F202740190ABD093D2A586
:10ABC600201002C2A512ACE08053C8A08269554687
:10ABD60046E536602324AA500AE53675F01984E561
:10ABE600F06027D2A6201002C2A6D2A57418304B58
:10ABF60002746412ACE08025E52B5403600C20102F
:0AAC06000E301106E54A64026005F5
:10AC100012ACFB800312AC5A101B08A25892A5A2DA
:10AC20005992A675A700D082D083D0A7D0F0D0E0EB
:10AC3000D0D020200C201009C5A6700302258BC59A
:10AC4000A632C218B40202D21812B995301808748C
:10AC5000E412D18B02AB6302AB5E78A7E5B4600966
:10AC600024E04005760002ACFBE534702920412247
:10AC700020751F300D1CE57924CE40167AFFE5B112
:10AC800010E7010A2325B3F5B3EA35B4F5B4C313CD
:10AC9000F5B2E660021622C241207502806DE579A8
:10ACA0006051206502C21CD265FF24B050027F4F64
:10ACB000EF90AD739375C70375C6FC75B90185BF79
:10ACC000F0A4E5F0F624F44002760C301C2DE5BE2D
:10ACD000C39FF5F0A4E5F024E0400375F020E5F013
:10ACE000C21C79AA770375B300F5B4C31375B1001C
:10ACF000F5B222C26578A77680D24179AA7703D2CD
:10AD00001CE4F5B3F5B4F5B1F5B222C265E57924DA
:10AD1000CE50097628301CE3743280C4768079A145
:10AD2000E720E7D7E5799740D279AAE7FAE57923D2
:10AD300023B4C500400274C42437300E30F42437E5
:10AD4000300D15F7BA0302FA0AC39AF5B175B300CC
:10AD5000EAF5B4C313F5B222101C06D21C76C880E3
:10AD600081763274FF200E02749B02ACE2C313247E
:10AD70007E80CDFFF3E8DDD3C9C0B8B0A9A29A9414
:10AD80008F8A85817D7975716E6B6865625F5C59AC
:10AD90005653504E4C4A48464442403E3C3A383660
:10ADA00034333231302F2E2D2C2B2A2928272625DB
:10ADB00025242423232222212120201F1F1E1E1D83
:10ADC0001D1C1CD2B5C28EAE8DAA8DAF8BAB8BE491
:10ADD000F58DF58BD28E3014012278B6BE0007EFC8
:10ADE00024E24002800806E624EC50027614206734
:10ADF00005E624F64005E4FEFAFFFB7C007D0A121E
:10AE00005BD27C007D5E125CF28F7EEE6003757E0D
:10AE1000FFEAFC7A33125BE6EBF5F0A4E5F0CB8CAD
:10AE2000F0A425E0C5F035E0CB926C25F050060B80
:10AE3000BB0002D26C30E7060BBB0002D26CECF513
:10AE4000F0A42BFBE5F03400FC306C010C78A6E696
:10AE5000C39BFF18E608F6EB18F618E69CFE18E60A
:10AE600008F6EC18F6301401227A0050040A125E3B
:10AE7000697C007D6E125CF28FF078A2E6A4FBACD8
:0CAE8000F0125E08EBBA0002F404FAE4E1
:10AE8C00F8FFEA30E70118E57960062075031FF436
:10AE9C00042AF579EF38D27520E70860037579FF3D
:10AEAC0002BBBDC2750470F5E579F40460EFF57969
:10AEBC0080EE120982E5BE78A2F624F65007E4F57E
:10AECC00BEF61248EE12097D85BC2B85BD21E5BE70
:10AEDC00F54824F65008E4F5BEF5481248EEE5BFF7
:10AEEC00F54324F3503924F3403512097878A1A6A0
:10AEFC00BCE5BF789DF61424FB50087403F6F5BF2F
:10AF0C001248EE78B7A6BE12096EE5BDA2E39266B2
:10AF1C00A2E49267035403C253B40102D2532274C5
:0AAF2C000DF5BFF5431248EE80C09A
:10005E0078FFE4F6D8FDF478D8F6F5A6D220D2B41F
:10006E00D2C075C07A75D75075AE1375AF01758154
:10007E00D87590F875EFBC75FDFFD2A412D0B9C239
:10008E00A4745012259E758951D28C75A882D2BC4B
:10009E0012AF3612D1B212B86D12AEBEC22012CC51
:1000AE00241224697F527E019090EE126C0C12483D
:1000BE004712D02612D0B912CE0812D02612D0E294
:1000CE007C1412D0C330000302258BDCF512439052
:1000DE00753A001243E2E53A701612D1E67F437E7E
:1000EE0006909756126C0C12D0263000FD02258B0E
:1000FE0075A6FF12439012AEBEC22B12246912D007
:10010E002612D0B512D0E278B5761E12CC2412B8D3
:10011E0062C215C21412246990910D7F78126BFA87
:10012E00205E0A7F767E1290911A12C7977F401238
:10013E00D0027F497E0978AEE612C6017E15743A6A
:10014E0012C7697E1AE53E12C6017E26743A12C7A0
:10015E00697E2BE53F20E00805A6E5A6700215A6F0
:10016E00E53F12C6017F5312BDD37F577E0B12C5DA
:10017E002E12C5B67F6030737F7E0BAC5DAB5C120A
:10018E00C53212C5B67E31126C977F697E1212CAC5
:10019E00BFE5A60303543FFDFE0D7F7312D12B0F57
:1001AE0012D12B1EDDF478B5E57124F64002761ED1
:0401BE00307419E69A
:1001C20060567F727E16744012C7377E17E612C6DB
:1001D200BF7E1F745312C73712D02610003710018A
:1001E2003710023712432ED2AC75369612CF35B481
:1001F200E00512442C800AE53670F112437E12D0DB
:10020200B20201192074097E2BE52E540712C7563B
:100212007E1702019502258B02278E8078E5352410
:10022200C8504FE59020E24AD0E0D0E012027502B9
:1002320057DBE53524D2503AE59020E235D0E0D0C4
:10024200E012D1E6803EE53524D25026E59020E248
:1002520021D0E0D0E012D1E6306B119093627F0999
:10026200126BFA12D02612492A12707E12027502FD
:10027200047E2212D1E69097D57F00126BFA12D03B
:100282002602D0B212D1E69097D57F00126BFA12F5
:10029200D02612D0B5C215C214C227C26812D0E24B
:1002A2007537019091B21217A09002AF730201014B
:1002B20002127B02066502199702047E0204BB0247
:1002C20057DB0202C712D0E27537079094FF12176C
:1002D200A09002D7730202970204F60205300205CB
:1002E200610202FB02036D0202C70202C702033768
:1002F20002031E0246A80203001243E580481218B8
:10030200F812D0261000BE10010280F89093627F8E
:1003120063126BFA12D02612AF9F80A91218F8123C
:10032200D0261000A010010280F812487312CC24CB
:1003320012AEBE80907F49A25E12082E925E120813
:060342004980821248EE22
:1003480012D0E27537029096BB1217A0900358732B
:100358000202C70209AD020A12020A69020ABE02B3
:100368000B02020B1112D1E69091527F017E091205
:100378006C0C90915A7F0A7E09126C0C7F1312BD87
:10038800CB751700120973E5BC12044DE5BD1204C4
:100398004DE5BE12044DE5BF12044D90919A7F5F62
:1003A8007E06126C0C12192C12D026751700120436
:1003B8002D10000810011510024880F20517E517E6
:1003C80024F7500375170075100080E2E5176408DC
:1003D800701512097375BC0175BD2375BE4575BFCF
:1003E800671248EE02036DE51012045F12D0261260
:1003F800040D0510531007E51724FE40035310039E
:1004080080AC0202C7A9BCAABDABBEACBFE517133E
:1004180004F8E640085407C42510C4800454702525
:1004280010F60272667800E875F009A42417FF7EBA
:10043800347D20E8651770027D71ED12C76908B830
:1004480009E502D026F8C4120453E812045F7E03BB
:100458000517E51702C756540775F007A49091626F
:100468002582F58250020583E51775F009A4241743
:10047800FF7E0C026C0CC26812D0E27537059092B0
:10048800DE1217A090049073020297026E4B026E60
:100498009002701F02047E0204B4026F61026FC7EB
:1004A80002124402047E02122A0207717F2E1211E0
:1004B8003580C312D0E27537069093A51217A09025
:1004C80004CB730202970212810212E302135A024A
:1004D80014270214590214D00204BB0204EC0215BA
:1004E800030215A87F4912113580C81248EE12D0B0
:1004F800E275370390956A1217A0900506730202F9
:10050800C7020792020DFC0207A70207B202119F59
:10051800020E83020855020EB7020EFD0211F10207
:100528000E6B020F421248EE12D0E2753704909615
:100538002C1217A0900540730202C70207C10207D8
:10054800CC0205300207E20207ED020B2B02053050
:100558000207FC0207D71248EE12D0E275370B905B
:1005680096711217A0900571730202C7020BCA0296
:100578000BCA0205980205D502056102056102123F
:1005880087020C56020D23020CC9020DB20208168E
:100598007F1C1209A512096EA8BE1205C912D02621
:1005A80010000810010D10021480EF18B800EB7845
:1005B8000B80E708E824F450E1780180DD88BE80EC
:1005C800957F1B7E35E875F005A402C6017F2512CC
:1005D80009A512096EA8BF12060712D02610000836
:1005E80010010D10021480EF18B800EB780980E7AD
:1005F80008E824F650E1780180DD88BF02055E7FB7
:10060800247E3BE802C756120991E5BF541F75F0D6
:0D0618003CA4ACF0FDE5BE75F005A42DFD81
:10062500E5F03CFC12096EE5BF1475F005A485BE26
:10063500F0A42DFFE5F03CFE7C007D3C125CFFC084
:1006450005EF75F01884E5F07F2D7E2412C6017E36
:1006550030743A12C7697E35D0E012C60102D02641
:10066500D25712D1E612188F1206730202977F171E
:100675007E02909204126C0C7F4C7E0290921B12AB
:100685006C0CAC5DAB5C7F577E0412C5AE12099154
:1006950085BC6285BD63E56124F840449092267F60
:1006A50037126BFAAE61AF607C017D5E125CFFC3F1
:1006B500741F9FFAAC63AB62EC3392175003125E62
:1006C50079125BE6AB047C00301703125E7974F592
:1006D5002BFB74033CFC125BBC7F377E1512C526D1
:1006E5009092337F697E0F126C0CE560240FFBE45A
:1006F5003561FCA25C923BD25C7E1E12C532A23BE8
:10070500925C7E30742012C7697E36742012C769E8
:10071500E5602562FBE5613563FC7F227E0412C539
:10072500AEE56245637016742E7E3A12C76912D023
:100735002610000D10011510022602069B7420805C
:10074500E81562E562B4FF0C156380080562E56291
:1007550070020563E53524F5500375330102069BE8
:100765001209918562BC8563BD0248EE1218F81224
:10077500D02610001510010280F87F637E05909346
:1007850062126C0C12D0261248F902047E12097806
:10079500E5BCA2E77F0A120837E5BC92E7F5BC0283
:1007A50004F37F1CA20D12082E920D80097F25A24D
:1007B5000E12082E920E1208490204F67F0AA20FA5
:1007C50012082E920F802A7F13A20812082E920873
:1007D500801F7F52A20C12082E920C80147F25A236
:1007E5000B12082E920B80097F2DA20912082E925A
:1007F500091208490205307F4912096EE5BDA2E3D9
:1008050012082E12096EE5BD92E39266F5BD02054A
:100815002D7F6D12096EE5BDA2E012082E12096E3C
:10082500E5BD92E0F5BD02055E12097D85BC2B850F
:10083500BD218F1F92171209A5AF1F1F7E39127890
:10084500D2A2172212097D852BBC8521BD0248EE57
:1008550020371412097885BE12120882120978858C
:1008650012BE1248EE80057F3F1208740204F67E20
:10087500039095F4126C0C12D02602D0B275A6FF27
:1008850012D1E612A96B740712D1D28FF074061239
:10089500D1D2EF2512C395F0FD78D8E6C4540F2DBB
:1008A500A2E7923D4010FD24CD50027D32AC05C338
:0B08B500743F9DFD800FF404FD24C87B
:1008C00050027D37AC0574402DFD7F4012BDCB7EBC
:1008D0001212D12B0EBE1EF91F303D020F0FEF6D0D
:1008E00070EDE536700A753606EC2513F5148C1399
:1008F00012090912D0261000071001083002072241
:100900001512800205120208827F377E28742E128B
:10091000C7697F347E21740A303D010412C786E521
:1009200014FC249C50027C63EC75F00A84C0F07FB8
:10093000347E2D12C786D0E07F377E3612C7567FB1
:10094000437E1E12C52E7E00E51212C6C57F057EAF
:1009500002909600126C0C7F6D7E0190960B126CCB
:100960003F7F747E0490961D126C3F02188F75C6EF
:10097000F6802B75C6F7802675C6F8802175C6F9F6
:10098000801C75C6FA801775C6FB801275C6FC8080
:100990000D75C6FE800875C6FF800375C6FD75C758
:1009A0000375B90122743F12C73702D0267F0A129D
:1009B00009A57E2A1243E5120982A8BF1209E11097
:1009C000001210010510021580F508E824E750EC2C
:1009D000781880E818E830E7E3780080DF88BF8087
:1009E000627F097E0590984DB80C03909847126C71
:1009F0000C7E27E53D28240C75F01884E5F012C61E
:0F0A0000017E33743B12C7697E35E53E12C60195
:100A0F0002D0267F131209A512097D85BC2B120A6D
:100A1F004610000810010510021780F2105C072025
:100A2F005D0BD25C80E8105DE5D25D80E1D25C8029
:100A3F00DD852BBC020345205C10205D189098A02B
:100A4F007F127E23126C0C02D0269098B4205DF09A
:100A5F009098A780EB9098AD80E67F1C1209A512A5
:100A6F00097DA8BF120AA010000810011110021A68
:100A7F0080F2E824F250031880EA780D80E6E8242B
:100A8F00E740030880DE781980DAE8F5BFF5438088
:100A9F00A37F1B7E26E412C756E82323B464087E87
:100AAF0026740112C756E47E2E12C60102D0267F8D
:100ABF00251209A512098CA8BCE8120AF912D02632
:100ACF0010000810010D10021F80EEE824E050E91D
:100ADF00188006E824CF40E10812098C88BC124820
:100AEF00EED21512CC2480D180157F247E3724E2DC
:100AFF0002C6727F2EA20A12082E920A120849020B
:100B0F0003487F3712096EE5BDA2E412082E1209C1
:100B1F006EE5BD92E49267F5BD0203457F367E1503
:100B2F00743E12C769120978A8BD120B9512D02610
:100B3F0010000810010510021080EFE82487500400
:100B4F00240A800224E8F880E17F367E29743E1261
:080B5F00C769120B9512D026A4
:100B670010000810011410022080EF18B80904784B
:100B77007880E7B878E478E780E008B87904780AFD
:100B870080D8B8E8D5787980D188BD02052DE824CA
:100B970087923DE8500224917F367E2FC313923B04
:100BA70012C6727E3CE4303B02740512C74F7E1AB0
:100BB7009099DB303D039099DF126C0C7F3C7E3AB5
:100BC70002D12B7F127E1F743E12C769120991A8AA
:100BD700BF53001F53BFE0120C3910000810010D5E
:100BE70010021480F218B8FFEE781780EA08E8249C
:100BF700E850E4780080E0120C397E2F743E12C76B
:100C07006912D02610000810011110021B80E81588
:100C1700BEE5BEB4FFE175BE0B80DC05BEE5BE24B4
:100C2700F450D475BE0080CFE8541F25BFF5BF022E
:100C3700055E7F127E24E812C6017E30743A12C721
:100C4700697E35E5BE75F005A412C60102D0267F80
:100C5700491209A5120C8CF853BF1F120C961000ED
:100C67000810010D10021280F218B8FF02780480F4
:100C7700EA08B80502780080E2E8C42354E025BFFB
:100C8700F5BF02055E120991E5BF54E0C403227F58
:100C9700487E059099F5126C0CE8601CB4040A7E36
:0F0CA700059099EA126C0C800C909A01126C0C5B
:100CB6007E38E812C75602D0269099FC7E29126C1F
:100CC6000C80F3120C8C60206404601C7F5B12099C
:100CD600A512097D85BC2B120CFE12097D10000B96
:100CE60010010810020C80EF020561105FE9D25F67
:100CF60080E5852BBC02055E120C8C601F640460C7
:100D06001B7F5A7E059099F5126C0C7E23909A05EE
:100D1600305F03909A0C126C0C12D02622120C8CA7
:100D260070030205307F521209A5120982A8BC126F
:100D36000D6112098210000810010810020880EFE8
:100D46001880EC0880E912098288BC1248EE120964
:100D56008CE875F005A4F5BD02055E120C8C604B9F
:100D6600E875F03270040475F028A4ADF0FC305D2F
:100D760011ACF0FB7A8A125BF4EB30E7050CBC0091
:100D8600010DAE05AF047C007D64125CFFC005EF6B
:100D96007F517E1A12C61E7E2C742C12C769D0E0B3
:100DA6007E2F12C601123CD412D026227F6412096D
:100DB600A5120982A8BD120DDF10000810010D1042
:100DC600021280F218B8FFEE787D80EA08B87EE657
:100DD600780080E288BD02055E7F63E82312C16F5A
:100DE60075F06484C0F07E2612C7567E2C742C12D1
:100DF600C769D0E080AA7F131209A5120978E5BC5D
:080E0600A2E7923DC2E7F8E803
:100E0E00120E3B12D02610000810010D1002128097
:100E1E00EE18B800EA783280E608B833E27801803E
:100E2E00DEE8A23D92E7F5BC79A1F78079547F30D8
:100E3E005C01237F127E2375F00A84C0F012C67205
:100E4E007E2D742C12C769D0E07E2F12C74F0F7EF5
:100E5E00359098BA305C03909916026C3F7F6412FD
:100E6E0009A5120982E5BE7F637E2C127927F5BE95
:100E7E0079A2F780317F371209A512097DA8BC53DC
:100E8E0000037F367E32E812C75612D026100008B5
:100E9E0010010710020780E718180880E2E5BC541D
:100EAE00FC48F5BCF52B0204F37F491209A5120983
:100EBE008CA8BE120EEE12D02610000810011110D2
:100ECE00021A80EFE8240AF8242450E778DB80E346
:100EDE00E824F6F8247F40DB788180D788BE80C670
:100EEE00E8F424DC75F00A847F487E3B02C7567F07
:100EFE00521209A512098CA8BF120F3512D0261056
:100F0E00000810011110021A80EFE82408F8245787
:100F1E0050E778A880E3E824F8F824A040DB786056
:100F2E0080D788BF020EB4E8F424A923C47F517E73
:100F3E003B02C7561226D0754A00D210C211D214E7
:100F4E00D27575791475340012D1E67F007E029049
:100F5E0095D5126C0C903CFD7F087E2612C797E546
:100F6E002B54030F7E3912C7561218AA12C3FF1242
:100F7E00833812D02610000810011A10022480C5E2
:100F8E00207504057980BE1579E579B4FF05C27523
:100F9E0075790180B02075EB1579E57970A7D2755A
:100FAE0080A3C210C2140204F612097DE5BE7F09A9
:100FBE007E3A02C756120982A8BF1209E112097DB4
:100FCE0085BC2B85BD21120A46A8BF120AA01209A4
:100FDE008CE5BC120AF97F2DA20A1210EA7F36A206
:100FEE00670210EA12097D85BC2B85BD217F1BA2ED
:100FFE000D1210EA7F24A20E1210EA120978E5BC37
:10100E00120E3B7F09E5BCA2E71210EAA8BF12112F
:10101E00DDE52B54037F367E3212C756120982E568
:10102E00BE7F637E2C12C75612098CA8BE120EEE1E
:10103E00A8BF120F3512096EA8BC02122212097D2A
:10104E0085BC2B85BD217F09A20F1210EA7F12A24B
:10105E00081210EA12096EE5BDA2E37F481210EAEB
:10106E007F51A20C1210EA7F24A20B1210EA7F2DE0
:10107E00A2091210EA120978A8BD020B9512099165
:10108E00A8BF53001F120C3912096EA8BE1205C953
:10109E00A8BF12060712060F12097DE5BE7F3F7E1E
:1010AE003A12C756120991E5BF54E0C403F8120C68
:0110BE00969B
:1010BF00120982A8BC120D6112097D120CFE1209D1
:1010CF0082A8BD120DDF12096EE5BDA2E07F6C8014
:1010DF000A12097D85BC2B7F48A25E744E400274B4
:1010EF00597E3A02C7691272727F73126F0E1272B3
:1010FF00C17F6C126F1D7F2D800E12097DE5BE7FA3
:10110F00097E3A12C7567F4812096EE5BD03540394
:10111F00F51075F005A47E1E9093762582F582500A
:10112F00020583026C0C1209A51F121117A81012C9
:10113F00111712D02610000810010810022780EF97
:10114F0018800108530003202B03530001C253B82A
:10115F000102D253E8235406F9E5BD54F929F5BD30
:10116F001248EE80CA22125A51EBF516F5147F6C15
:10117F00126F1D125A357F647E23E51612C6D5C332
:10118F00E5169514F5167F73126F0E7F2D0211174A
:10119F007F2E1209A5120978A8BFE824FA40033060
:1011AF00370278031211DD12D02610000810010D3E
:1011BF0010021280E518B800E1780580DD08B80646
:1011CF00D9780180D5799DE8F7F5BF0204F37F2D1B
:1011DF007E2C7420B80502742E12C7697E32E80285
:1011EF00C7567F5B1209A512096EA8BCE81212221E
:1011FF0012D02610000810010D10021280EE18B840
:04120F0000EA780376
:1012130080E608B804E2780180DE88BC0204F37F2C
:101223005A7E2CE802C756D26875480A1243E5D2A3
:10123300141225D31273AC122F1FC26B12024880F3
:10124300F3D21475150112722C75B901E5BC20E7B0
:101253001C12735C75A6FF1273B81218B512D02650
:10126300126D1510000F5005126E3D80E70515E550
:1012730015242050D102047E12128D0202971212FD
:101283008D0204BB12128D02056112129912097D9F
:101293008548BE0248EE1225C51225DF12628C1264
:1012A300D1E6909408D249127C04127BBD121865D2
:1012B30012D02610001410010510021B80F50548FA
:1012C300E548640A7002F54880CF1548E54864FF95
:1012D300700375480980C28548491225DFE5582205
:1012E3001243E51225C5854849C250E558B40F029B
:1012F300D25012628C8038D22775480A1225D31235
:10130300628C12D1E6127B2C90979C202903909734
:10131300A7121919C26A122F1F106A0280E1C2278D
:101323001272048549481216D71225DF12628C12F5
:10133300D1E6909345127C0220500E12190312D06D
:10134300261000101001B080F81218B512D0261024
:10135300000280FB0204BB1225C5E55830E7137F6A
:101363001B9097867E05126C0C12D02612D0B50204
:1013730004BB1225DF12628C85594912D1E612187B
:101383009F9097A7127C02127BC712D026100008E9
:0D13930010010A10020C80F51213F280DB2D
:1013A0001213FF80D612D1E612189F909418127C67
:1013B00002127BC7127BCB12D02610000810010A44
:1013C00010020C80F512140B80DB12141980D61257
:1013D000169D1225DF12628C12D1E6909709127CBD
:1013E000021218DD12D02610000510028880F802C3
:1013F00004BB0559C3E5589559500375590022158A
:1014000059E55964FF7003855859220549D3E549C8
:101410001495584003754900221549E54964FF7049
:10142000058558490549221225C5E55830E7057F4D
:10143000240213641225DF12628C12D1E6909423E9
:10144000127C0212190E12D02610000A100102801E
:10145000F812174680DE0204BB1225C5E55830E7B6
:10146000057F2D021364C26B7559FF12628C12D175
:10147000E612188FE55930E7031218AA9094341237
:101480007C02127BD712D026E55820E70610000810
:1014900010011110021B80F00559C3955950CF75EA
:1014A00059FF80CA1559E55964FE70C285585980A4
:1014B000BDE55920E711D26B75A700758307C4F508
:1014C00082E0B2E7F080A7306B031216F40204BB8F
:1014D0001225C5E55830E7057F360213641225DF73
:1014E00012628C12D1E690943F127C021218F8120C
:1014F000D02610000B10010280F812173B12177053
:101500000204BB1225C5E55820E7087F5190944995
:0915100002136712D1E69097B2B4
:10151900127C021218B512D02612431ED2AC10004A
:101529001FE55830E7F8306DF512163D7E207F0033
:1015390050139097CB126C3F12D02612D0B580CAA7
:10154900C2AC0204BB1B8B13909362126C3F12D086
:1015590026C26B7B007514B812173012732B1272E6
:10156900DD5025A814E824384004A60105140BC34E
:10157900E5139B50E678B8121772306B0312707E30
:101589001225DF12628C8082127272E51660E6D231
:101599006B127388C003127243D003A91580C41259
:1015A90025C5E55830E7057F5A0213641225DF1275
:1015B900628C12D1E6909454127C021218D212D085
:1015C9002610003510010280F875460512160550DF
:1015D900157F007E357407954612C6D512D026129E
:1015E900D0B5D546E7D39097BD50039097CB127CE1
:1015F9000212D02612D0B580B30204BB12431E12C8
:10160900CDD0745212CE03745412CD9EE558047590
:10161900590012CDBF126CC4401612720412735CC9
:10162900126D15400B0559C3E558955950ECC32265
:10163900C2ACD32212431ED2AC12CF30204CF1B42B
:1016490040F712CF35B4400312CF35B452E2F53822
:1016590012CF35B454DA12CF35FA60D424EF40D022
:1016690012CF35E53870C912CF3512CF35126CA9B2
:0F1679007B007E03126DA050102050B412CF35AD
:10168800204C03B440F7DEED80A712733B0B126CBD
:10169800A9DAE0C322121781E55924C8F88602E5C1
:1016A8004924C8F9986013146010500F18E608F61A
:1016B80018E86970F7A70212177022E559640F60DD
:1016C800F91908E618F608E86970F7A70280E81221
:1016D800178178C8C250E6B4FF02800708B8D8F668
:1016E800D25022B8D702D250A615807C78B81217EB
:1016F80083E4F9F5A7758307E9C4F582E030E70AC2
:10170800E924B8F82438400276FF09C3E55899500F
:10171800E712173B78B879C8E6B4FF028002F709E8
:1017280008E8243850F2804079B877FF09E924386E
:1017380050F82279C877FF09E9242850F8221217AF
:1017480081C23D78D7B6FF04A900D23D18B8C7F5C5
:10175800203D0279D81978C8B6FF0122C3E899500C
:1017680007C6C7C6081980F478C812179212739A68
:1017780012739A12739A02739A78C8121792127394
:101788007612737612737602737675C703E5487519
:02179800F0045B
:10179A00A42480F5C62212D1E6C23C126BFEE537BC
:1017AA00604E14604814604014603814603014604D
:1017BA002814602014600E14600B14600D14600568
:1017CA0014600C802B1210E08026121175802112F1
:1017DA00108B801C12110980171210F5801212103A
:1017EA004B800D120FF28008120FC38003120FB73D
:1017FA0012D02612D0B912188F12AD01A81F08E80C
:10180A0014C23BB51D02D23B75F007203C0375F0AC
:10181A0009A4FF7E00303C0C7420303B02743E1257
:10182A00C737800A740B303B02740A12C74FD8CFED
:10183A0012D026E51D10000810011010021880B9F8
:10184A00651F7003751DFF051D80AE7005851F1D80
:10185A0080A7151D80A375F003A4227F7B7E0090CC
:10186A00996E126C3FE54824F640087E0A90976804
:10187A00126C3F22126F3A7E05745B12C7337E1DCB
:10188A00745C02C73312187E7E3490997F026C3FD3
:10189A00126F3A800312187E7E31909983026C3F50
:1018AA0012187E7E319097D6026C3F126F3A7E00F4
:1018BA008005126F3A7E2D9097D6026C3F1218D28D
:1018CA007E3190938A026C3F1218B57E1A90938FDC
:1018DA00026C3F1218B580C01218B57E1890934F4B
:0618EA00026C3F1218B56C
:1018F0007E1A9097DB026C3F1218B57E1A9097E023
:10190000026C3F1218B57E1A909412026C3F1218A6
:10191000B57E1890942E026C3F7F007E20126C3FA3
:1019200002D026126F3A9097E6026C3D126F3A9001
:1019300097F7026C3D12B1DB12099BE5BDF55EF530
:101940006CE5BCF55FF56B756A007561FF75A70402
:1019500090070012B187B4FC12E582C313F561E56C
:101960006CF0E56BF0E58260168005B4FF02800F35
:1019700012B0D6E56C655E70DAE56B655F70D475A4
:10198000A70022E560758307C333F582E0A3F56CF9
:10199000E0F56B756A0022D214C21F12193575600A
:1019A00000E561B4FF1612D1E69092367F0A7E05FB
:1019B000126C3F12D02612D0B2020297C210C2118E
:1019C00012D1E612188F301F0A7F07909244126CD2
:1019D0003D80647F007E01C3E56012C6D57E0E7433
:1019E0002812C7338560487407F51FFF7E00743ED8
:1019F00012C737E54812198512BBD9121F1E0548B8
:101A0000C3E5619548FD401CE51F2407F51F24C868
:101A100050E17F387E01ED0412C6D57E0E74291286
:101A2000C733800DE51F2407FF7E019097D5126C08
:101A30003F201F03121F6112D02610001910012C25
:0B1A400010020280F5120234301F3D3E
:101A4B00020286101F02D21F0219BCE56160F4E589
:101A5B006065617005201FF080E9201FE60560803E
:101A6B00E7E56160DEE56065617005201FD58009E3
:101A7B00201FD5E560700280CA156080CB12193526
:101A8B0012198312BBD9122055756A1012B16E123E
:101A9B00210C90924BD23C126BFE121800901AAC98
:101AAB00730219BC022D76021AD5021AB81218F855
:101ABB0012D0261000C710010280F812198312B140
:101ACB0087C2E2FF12AF85021997C2531219831214
:101ADB00BBD97537009092641217A0901AEA730263
:101AEB001A88021CD7021CDC021AD5021B11021B1E
:101AFB0016021AD5021B54021B58021B5C021B63F5
:101B0B00021B67021B6B12434B8003124336780A8E
:101B1B00121C34740712CD9C121C7312CDB8121CFC
:101B2B00AE12B16E12B19A12B09712B2B1121DC8A9
:101B3B00D5150C75150A121CC1121EE812CDB81062
:101B4B000204E57F70DB021A88780A80067804802D
:101B5B0002780112434B800D780A800678048002CC
:101B6B007801124336121C34740712CD91121C7378
:101B7B00E54812CD7D742A12CD9E12CD9E12CD9EBC
:101B8B0012CDB8121CAE12B16E12B19A12B09712DE
:101B9B00B2B1121DC8D51548854815121CC1E51CDC
:101BAB0012CD7DE51B12CD7DE51B2548F51BE435DC
:101BBB001CF51CE4A27792E7A27492E0A27392E167
:101BCB0012CD7DAD75AC74AB73E57DC4121BF5AD59
:101BDB0078AC77AB76E57D121BF5121F0612CDB8EC
:101BEB00100204E57F709F021A88540F2375F005CD
:101BFB0084F8C3EB33FBEC33FCED33FDC3EB33FB6E
:101C0B00EC33FCED33FD20E713EB28FBE43CFCE469
:101C1B003D12CD7DEC12CD7DEB02CD7DC3EB98FB60
:101C2B00EC9400FCED940080E888481218BCE4F5B5
:101C3B004AF549756A2075150112B16E12B097D528
:101C4B00150E854815E5492401F549E4354AF54A51
:101C5B00E57F70E5744012CE03747812CD9E7463E9
:101C6B0012CD9E741F02CD91121EC3E56012CD7D65
:101C7B0012198312BBD9E53A12CD91E53B12CD91E6
:101C8B00E53C12CD91E53D12CD91E53E12CD91E5AE
:101C9B003F12CD91740112CD7DE54A12CD7DE54900
:101CAB0002CD7D121983756A20E4F51CF51BF51422
:101CBB00F51375150122753800E51412CD7DE5136A
:101CCB0012CD7D0513E513700205142212434B80D0
:101CDB00031243211218BC121E1E12D0BD756A20AE
:101CEB0075150175A6FF754A0112B11212B0971244
:051CFB00B2B1121DC88A
:101D0000D5150975151E121DEC12D0C7121EE8E577
:101D10007912CD7DE57EB47F01E4C333500274FFB8
:101D200012CD7DE571121DAD12CD7DE57012CD7D18
:101D3000E57B24ACFFE55F340912CD83EF12CD7D46
:101D4000E51520E033857D56E412CD7DE52EC412E5
:101D5000CD8312CDC712D0C710021A3055907440EF
:101D600012CD9E744512CD9E744F12CD9E744612B4
:101D7000CD9E12CDC7021A88E556121D87C4FAE51A
:101D80007D121D872A80C2FBC4121D942323CB120F
:101D90001D942B22540FFC24F650027C00901DA3AE
:101DA000EC932200000101010202030303FA244024
:101DB000400A24804003EA3322D2E72274FF222023
:101DC000E703C3132224C022E53F701F7F7B7E0000
:101DD00078AEE612C6BFEE2404FE743A12C737EEA0
:101DE0002404FEE53E12C6B912D02622C015D21236
:101DF000129A44C212D01578AEE612CD91E53E1289
:101E0000CD91E53F12CD91E54512CD7DE55212CD44
:101E10007D740A12CD7D74C012CD7D02CDC7744091
:101E200012CD9E745412CE03744E12CD9EE412CD88
:101E30007D121EC3741F12CD91E53D12CD91E56058
:061E400012CD7D12198392
:101E460012BBD978ABE60812CD91E60812CD91E621
:101E56000812CD91E612CD91E53E12CD9112245095
:101E6600E51212CD91E51112CD91740112CD7D903E
:101E76009808121F10756A1012B16E057F057F78DB
:101E86007F12CD76787B12CD76787D12CD767877F7
:101E960012CD76E4FEFF780712CD7612CD76E57484
:101EA60012CD7DE57512CD7DE412CD7DE573C3338C
:101EB600500274FF12CD7D12CD7602CDC775C703D1
:101EC60075C6FF75B901C217751D0085BC1C85BD99
:101ED6001B85BE1A85BF19125B6CEE12CD7DEF0213
:101EE600CD7DE57512CD7DE57412CD7DE57312CD00
:101EF6007DE57812CD7DE57712CD7DE57612CD7D37
:101F0600E55E12CD7DE57A02CD7D75A700E493707E
:101F16000122A312CD9E80F5AF1F7E0478ADE61296
:101F2600C6B97E0C742C12C7377E0E18E612C6B9D7
:101F36007E1A78AEE612C6B97E22743B12C7377E89
:101F460024E53E12C6B97E2FE54012C6BF7E377421
:101F56003B12C7370E0EE54102C6B975320012199B
:101F66008312BBD9857946787A796412BBF2746498
:101F7600125F478E47122055756A20D23D12B16E08
:101F860012B19A12208C303D09307406C23D8E1E65
:081F96008F1FE57F602BE54C75
:101F9E0024FFF54CE54D34FFF54D454C600512B070
:101FAE00AC80D2751D3C12B16E12B19A12B097125E
:101FBE00208CE57F6003D51DED1220ED90210512DA
:101FCE00C797203D0DAE1EAF1F1220ED9020FE12C2
:101FDE00C797E546FD700B90993E305D1190993A8A
:101FEE00800C04701090993A305D039099367F38CA
:101FFE00123CCE804BE4FFFC7E05305D047E027FFA
:10200E00B3125CF2AC06AB07125BBC7F38C23DE587
:10201E001C6007D23D7E2C12C724E51B203D0260BA
:10202E0007D23D7E3012C724E51A203D026007D24A
:10203E003D7E3412C724E5197E3812C724123CD3D4
:10204E00E53224C850FA22E54075F03CA42541FF44
:10205E00F54CE435F0FEF54D7C007D10125CFF0F63
:10206E008F4BAF4CAE4D7C007D3C125BD27C00ADF5
:10207E004B125CFFEE4F70010F8F4C8E4D22786429
:10208E007973C2D11220A3FF78677976D2D112204C
:10209E00A3FE02D12BC3E796FB0809E796FC0809BD
:1020AE00E796FDA2E792175003125E8175135A3020
:1020BE00D10E751320B217AA47125C06AB04AC05FD
:0720CE00E546600B04600B06
:1020D500AA46125C1DEB03FBEB03FBEB543FFBE550
:1020E500132B2017029B9B22EE141430E701E4FE0C
:1020F500EF141430E701E4FF2205057088A8887005
:1021050005052020F8202075320012D1E67E1E7FBD
:102115001C12D12BDFFB12D12B7E1E7F1C12D12B63
:10212500DEFB7E1D7F1D12D12BDEFB7F007E21781D
:10213500ADE612C6B97E29742E12C7377E2D18E674
:1021450012C6B97E35742E12C7377E3918E612C607
:10215500B97F077E21745412C7377E25744F12C785
:10216500377E2D78AEE612C6B97E35743A12C7377A
:102175007E39E53E12C6B978AE1224507F0E7E2117
:10218500744C12C7377E25744112C7377E2DE51270
:1021950012C6B97E35743A12C7377E39E51112C6B3
:1021A500B97F157E25744412C7377E2DE54012C6CA
:1021B500BF7E35743A12C7377E39E54112C6B97FFD
:1021C5001C7E2F85715412C23E7F217E0190990994
:1021D500126C3F7E0EAC77AB7612C56B7E2B857984
:1021E5005F85787B12CB187F287E0190990D126C44
:1021F5003F751D2B751E10E5741224047E25742F62
:1022050012C737751D2D751E2BE5751224047F2FFA
:0F2215007E02909901126C3FE57360031222B1B3
:102224007F367E029098F9126C3FE5721222B11249
:102234002349121983756A209004E6E56CF0900432
:10224400E7E56BF0AE4DAF4C7C007D40125CFFBF08
:1022540000010F0FAC07AD07E4FED23D12B16E12C0
:10226400B19A1222F2E57F602CE54C24FFF54CE58F
:102274004D34FFF54D454C600512B0AC80DE751D44
:102284003C0E12B16E12B19A1222F7E57F6006126B
:10229400B097D51DED1222C77F7812BDDD7F767E03
:1022A40000743012C737E53224C850FA227E211256
:1022B400C16F12C6D57E2F909911305D0390991687
:1022C400026C3F9004E6E0FD9004E7E0FCC3E56A9D
:1022D4009420FBE56B9CFCE56C9DFD50032410FDF4
:1022E400125DF19004E8EEF09004E9EFF022DD03D2
:1022F400AD040E7F78E55E20E72AE57A8549F0A4EF
:10230400A9F0E57A854AF0A429F9E435F0FAE55E06
:102314008549F0A429E435F02AFAE55E854AF0A45B
:102324002ACF9FFF12D12B103D18C3EF9B50131BD4
:10233400EF6B600E8F018B0712D12B1FEF6970F8C2
:04234400AF01AB0733
:10234800229098BE305C039098D7754A4075490032
:10235800AF76E577FE20E76B7005EF24105064EF49
:1023680024A8EE34FD40119098C3305C039098DBAC
:10237800754A1975499A8075EF2450EE34FB40115F
:102388009098C8305C039098E0754A0C7549CD80E8
:102398005CEF24A0EE34F640119098CB305C0390AB
:1023A80098E5754A067549668043EF24F0EE34F1E6
:1023B80040139098CE305C039098EA754A047549AA
:1023C80044802A8028EF2490EE34E840119098D178
:1023D800305C039098EF754A0275498F800F90988A
:1023E800D4305C039098F4754A0175499A7F40127D
:1023F8006C3D7F4612BDDD7F5F02BDDDAE1E75F010
:1024080064305C0375F03284C0F0F87004EE240484
:10241800FEE51D12C737EE2404FEE8600712C72444
:10242800EE2404FED0E075F00A305C0375F00584F4
:10243800A8F012C724EE2404FE742C12C7370E0E1F
:10244800E8305C012302C724E53E2541F51124C488
:102458005003F511D3E63540F51224E85002F51281
:102468002212ACFBC21012D1E67F057E099090E5DE
:10247800126C0C7F137E0890249D12C7977F2B7EC9
:072488000190250512C79722
:10248F0020370A7F277E2790257712C79722113092
:10249F0007FE1FE001E101F80F00061B00F80C001A
:1024AF00180E007C10007006003C2000E006003E75
:1024BF004001E004001E8003C004001F0003C0049D
:1024CF00000F00078000000F800780000017800FAB
:1024DF0000000027C00F00000043C00F0010008352
:1024EF00E00F00200301F00700C00F01F803830085
:1024FF007F87FE01FC000E3E180000030000000065
:10250F001800000300000000380000000000000069
:10251F003000000000000000FC761F0E1C6030EC45
:10252F00FCBC3F172DF0F978613866264F619A7021
:10253F006070C60E1EE330E06060C60C1CC360C046
:10254F00E0618C0C18C7C0C0C0E18C1C39C611C02B
:10255F00C4C19C9931963180C8C1FF1E31E7E1801B
:10256F00F0C0EE1C31C38180061630918828928806
:10257F004924904927909248A0E3C8BCC2AFD2C06B
:10258F0075C0107581D874FE12259EC2B480FCD21E
:10259F00A6C2A512ACE012D0B902AD0175C703E512
:1025AF004875F004A42480F5C6C23C75B901E5BC9A
:1025BF00047002D23C2212097DE5BEF54824F65084
:1025CF0003754800753400753704C228D229D22A02
:1025DF0075C703E54824E75003754800E54875F0D3
:1025EF0004A42480F5C6751607751700C23C122681
:1025FF0020122620122620122620851758155875CE
:10260F005900E548B40A09E5586005F46002055918
:10261F0022203C1D75B90105C6AABCABBDACBEAD31
:10262F00BFEA122641EB122641EC122641ED12268B
:10263F004122203C07F515B4FF03D23C22C0C7C08E
:10264F00C612722C75A704851683E517C4F8F58298
:10265F0075B90105C6E5BCF0C582F82406F9240357
:10266F00C582E5BDF0E5BEF0E5BFF075B90105C661
:10267F00E5BCF0E5BDF0E5BFF08516838982E4F097
:10268F0075B90105C685BC1385BD14E4F0F08882C9
:10269F00E5BEF0E5BFF075B901E5BCF0E5BDF0E5CD
:0526AF00BEF0E5BFF0E4
:1026B400758306E51723541E24B0F582E513F0E56F
:1026C40014F075A700D0C6D0C705172212AEBE7885
:1026D400BEA64808E4F6F55908761808F6D2360876
:1026E400760A08F6060876BEC225C254C25512B14F
:1026F400F01225D3C229C22AC207C227C268C24324
:10270400C24AC246E4F52EF534F536F52F78A8F61C
:1027140078B6F678B5F678A9F6789EF678B8A65E17
:1027240008A67A12C4D4C26BC233C238C240C223D0
:10273400C22212275E75460278C5A646C23AD22145
:10274400C219C22685705778BA7401F608F608F6DD
:1027540008F6E4F542F541F54022E45407205E0909
:10276400B4040040027403801B120973C313A9BC90
:10277400600C14A9BD600714A9BE6002A9BFE9409A
:1027840001C45407F53722020101754E501226D0B8
:102794001279F37544031243E212A26BD544030287
:1027A400258B201EF1789F7680754A0012AFDED209
:1027B40010C211C213C21212432E75A60C12CC24DD
:1027C40012B862E5A624FA400612437E75A60C20D0
:0427D4002517E59050
:1027D80020E206E5352405400CE59054057009E52E
:1027E8003524E2500302288AE5322418400D75F09A
:1027F8000C84E5F070C9122F2280C4D21ED2AC30EE
:102808006DBD7532F012CF3AB4E0B412442CE53104
:1028180024F39205201203122CC6122844C0141265
:10282800827ED014122991122F22129A1312B3E920
:10283800122F221279F6122F220227BB30123AE504
:102848004024F040257A0AC3E53F954B601C402A96
:1028580024E24016E53F453E7003757E7F305405FF
:10286800C254757F0112B008DADDE5510404F57F22
:1028780024FE4003757F02C27722F40424E250EA62
:1028880080D212D1E67F2A7E0E90980C126C0C75BD
:10289800A6FFC2101012137F367E0890936D126C3B
:1028A8000C12D02612D0B2020101D2211244061213
:1028B800B0127F1E7E0B909760126C0C12D02612FD
:1028C80028DD7F3E7E079094DD126C0C12D0261214
:1028D800D0AC02258BD215D22012B1C712097D8542
:1028E8002BBC8521BD75B90575B90212B1D1D25578
:1028F80012B0D07F0012AF85D22012B1D1E56A6044
:102908000512B09780F7857A62D22012099B85BE9E
:10291800BC85BFBD856BBE856CBF75B90575B90231
:1029280085BD6C85BC6B756A2012B1C7122B361237
:10293800B10412B1D1756A0012B16EE57064FE700F
:01294800434B
:102949007570FC854077854178851F797818797A83
:1029590012BBF212B0417FB412B0F0D22012D0C72C
:1029690012B1D1756A1012B16E8554717F08781051
:10297900797212BBF485627C855E7D12B0417FC499
:1029890012B0F0C220C21522300A012212434B12A2
:102999002AE2745212CD9E744D12CD9E744312CD0B
:1029A9009E122AF112CDD97441207402745612CDA7
:1029B9009E122A3E122A8812CDD9E53C12CD91E504
:1029C9003B12CD91E53A12CD91122ABE12CDD9749E
:1029D9004512CD9E122B27122AE2744712CD9E74FE
:1029E9004712CD9E744112CD9E122AF1122A3E122F
:1029F900CDD9E43074010412CD9C12CDD99004C311
:102A0900E012CD9112CDD99004E4E075F00A84AFBB
:102A1900F012CD9112CDDDEF12CD9CAC5EAB7A12E6
:102A29002B03AC5DAB5C122B0312CDD912CDD9129D
:102A39002B2702432E7875C23D122A497878D23D58
:102A490012CDD91276D8303D05E51E12CD9CE51D73
:102A590012CD9C122ACBE51812CD9CE57D203D01B3
:102A6900C4540F12CD9C12CDD9303D09744530178D
:102A79000274578007744E301702745302CD9E209A
:102A89007408122ABE122ABE802775A7049004BFB3
:102A9900E0FCE0FB7A1B125BF47832125D96125B64
:102AA900BC122AC89004C1E0FCE0FB125BBC122AEC
:042AB900C875A70035
:102ABD002212CDD9E4F51AF519800D12CDD9E51CE8
:102ACD0012CD9CE51B12CD9CE51A12CD9C12CDDDCD
:102ADD00E51902CD9C742412CD9E744712CE037459
:102AED005002CD9E12CDD9E53D12CD91E53E12CDD0
:102AFD0091E53F02CD9112773412CDD9E51D12CD5E
:102B0D009E781CE612CD9C18B817F812CDDDE41294
:102B1D00CD9C12CDD9744D02CD9EC038742A12CDE4
:102B2D009ED03812CDB802D0C778107F0EE4F608CB
:102B3D00DFFCF564F565F567F5687515FC751AC06C
:102B4D00751DC0756640756940754A0112B1123028
:102B5D005503022BF612B097E571B510004002F542
:102B6D0010E57EB47F01E4B511004002F511E512C8
:102B7D00207502E513C395795006207545857913A7
:102B8D00D3E57A9514E5156480FFE55E64809F407A
:102B9D000C857A14855E15857B16855F173074A9B3
:102BAD00C2D178647973122BD478677976122BD4CD
:102BBD00D2D178187973122BD4781B7976122BD445
:102BCD00808785791280B9D3E7960809E7960809B9
:102BDD00E66480FFE764809F20D101B3400AE7F6E9
:0B2BED001819E7F61819E7F622E51AA0
:102BF800B4C00E7873791812BBF27873796412BB7B
:102C0800F278187964C2D1122C677418125F478E53
:102C180047AE1EAF1F781B7967D2D1122C67C3E568
:102C28001F9FE51E9E50048E1E8F1F7EFF7FFFACE8
:102C38001EAD1F125CFF7A04EF8AF0A4E5F0CE8A7D
:102C4800F0A42EFEE435F0BEFF011E6005146005F9
:102C58007EFF8E1F22EE7E0020E7F77EFE80F3C304
:102C6800E697FB0809E697FC0809E697FD18181986
:102C78001930E703125E81C3EB33FBEC33FCED3311
:102C8800FDEB33EC33FBED33FC30D105AA47125C86
:102C98001D0BBB00010C751E03751FFFEC24FC40C7
:102CA800048C1E8B1FE627FB0809E637FC0809E69B
:102CB80037A2E713F618EC13F618EB13F6221013E5
:102CC8001978B5E624FA401AE57124F64008E57942
:0F2CD80024F6400280380606803412D0C3E590FF
:102CE70030E2DFD220753612D22EE4F534F55A12CF
:102CF700B222122D1CC219C25712275E1285C112A9
:102D070085EED212853F4B754C00205E02D2281209
:102D17002748C22022D214122D6BE6F008DFFB856C
:102D27007A62122D617570FE783A797112BBF212D0
:102D3700B041122D6185627A855E7B12099185BC4F
:102D47007E85BD7F7570C012B041122D6BE0F6080D
:102D5700DFFB75A700D254C2142274FF7870F608FF
:102D6700B880FB2275A7049004F078707F102212B8
:102D7700198312BBD912B33E9004EAECF09004EB2E
:102D8700EBF0124321751F03121E1E12D0C3D51F6D
:102D9700F71226D012D1E612D026C258C259756A48
:102DA7002012B112125F458E47754A01753901C26B
:102DB70010D211D214D21212B2221285C11285EE8C
:102DC70012CC2475A6FF753609753200E59020E20E
:102DD70006E5352405400CE5905405701FE53524BC
:102DE700E25019C211C21212D1E612D026E4F5350B
:102DF700F52F7E0612D0BFC202021A88E54A20E0EC
:102E07001612B32112432112CDD0744912CE037882
:102E17000412CD7612CDB8C221E54AB40202D221FE
:102E270012B112129A1330260F1262EE1279F6754A
:102E37003606E53670FCC2261279F3122F22E54AD0
:092E470020E022B4020A753900F2
:102E5000E53670F9022DC7E53960F9FD24E240023C
:102E6000053912B1122026C8DDF880E87539001244
:102E70004321D2ACE536602712CF35B440F612CFED
:102E800035B4400312CF35B44915F53812CF65FC7F
:102E900012CF65FBAD3812CF656D7003122EA3C241
:102EA000AC80B1C39004E9E0FF9B9004E8E0FE9C95
:102EB00050048E048F038C148B137A10125BF474FD
:102EC000202BF56A9004E7E03CF56B9004E6E03DCA
:102ED000540FF56C754A0112B112AE14AF137C0E8B
:102EE0007D10125CFF8F40AE04AF057C007D3C126C
:102EF0005CFF8F418D429004EBE02513FF9004EAC4
:102F0000E03514FE7C0E7D10125CFF78AEA607AE95
:102F100004AF057C007D3C125CFF8F3E8D3F227527
:102F2000370410003A100116100216E52F540760FE
:102F30000312ACF520783D20790A207A1F22023155
:102F40000B02306EE5376009146009146009023124
:102F500094023127023165C2790231B1023092E523
:102F60003724FC500FE5376407600302322C02312E
:102F7000F00230382011FAE59020E20280587534D2
:102F800000201203D2132278A9E67019C226767D9A
:042F9000E5377005AC
:102F9400106B02D26BD277D24A753614D22E02B29B
:102FA40017E5376043146040B40227200B24E6245D
:102FB4009B401F2414501C1285C19097337F207EA0
:102FC40008126C0C12D026753608D22E78A9E62485
:102FD400ECF622241940FB241450F71285C1128503
:102FE400EE90973C7F2980D72028E7E54824F640D7
:102FF400E1E5580460DC7F5D7E10E6249B40D32429
:10300400145015C2330559C3E558955950058558D0
:1030140059D22690972180A9241940B6241450B27D
:10302400E55960021559102606E5596002155990B4
:10303400972A808D10780122753900E534243840B0
:1030440007754A0175340022700AE54A30E0F275CA
:103054004A0280F0146008754A061285EE800675EF
:103064004A041285C175390180DA302909C229D28E
:103074002A7559008005302A0CD229127BB3127BA1
:103084008175340022206841302703D26A22D2227B
:103094001233C812D026107A0122E53424384007AE
:1030A40012275E75340022700FAA3712275E6A70E9
:1030B400F2740112275F80EB0412275F24FC50E3B3
:1030C400E537B40706D22880DA8036C228E53724EB
:0730D400FC2324BEF879C4BF
:1030DB00E7F9A74809A75979C4E8F786480886078E
:1030EB00E537B40505754818D2361225DF8F59E53B
:1030FB003764067002D2070230A71233A402334E94
:10310B00E537601814605314600C14607CE53724A9
:10311B00F940060232A60231DF023273D223123B90
:10312B00B910790122E5342438400775460175340E
:10313B000022700EE54624FE40F1E54660ED154693
:10314B0080ECB40500500C04F54624FA50E07546AB
:10315B000580DB100FD8D20F80D4D223E53464C89E
:10316B006003123BB910790122E534243750097002
:10317B0011105B32D25B802E100802D208123BB9C1
:10318B008024100C21D20C801DD223123BB9107954
:10319B000122D24BE53424374010C258C2592011BA
:1031AB0005D22E7536077534002224FD40152403F5
:1031BB007006D258C25980EEC258D2591460E7D269
:1031CB005880E3120978E5BCB2E7F5BC79A1F71298
:1031DB0048EE80D278B8A65E08A67A2011C875365C
:1031EB0005D22E80C130122B127BED055BE55B7592
:1031FB00F00B84E5F0F55BE55A24F64009E55A95AA
:0E320B005B5003755B00127BF112D026E53498
:103219006003D534D275340022D229D22A75480ADE
:10322900023314C2401007F1302903023314127B10
:10323900AF127BC3102A1BC2330559C3E5589559F0
:1032490020E7025008755900E548B41816E558B446
:10325900FF03755900127BD712D026E5346003D5D8
:1032690034C122D22A127BB380EE301223127BEDB5
:10327900155BE55B30E70C755B0AE55A24F64003FC
:10328900855A5B127BF112D026E5346003D534DA16
:1032990075340022D229D22A754817804CC24010B1
:1032A90007F2202944127BAF127BC3102A22C233B2
:1032B9001559E55930E71C855859E558B4FF037588
:1032C9005900E548B41802800AD22A127BB3800E4D
:1032D900855859E558B4FF03755900127BD712D0A8
:1032E90026E5346003D534B52220106220115F7FB2
:1032F900180548E54864187008F5483027037548EB
:103309000A1225AB303C2DDFE8802620105A201107
:10331900577F181548E54830E705754817800A644E
:103329000970063027037548171225AB303C05DFB5
:10333900E275480A1225DF12628CE532244C5005E9
:10334900127B818003127B2C75340002D026123344
:103359008B7F15E5486B70048A4880020548122561
:10336900AB303CD0DFED80CC12338B7F15E5486A5A
:0E33790070048B48800215481225AB303CB61C
:10338700DFED80B27A007B09E537B40401227A0ABF
:103397007B17B40601227418FAFBF5482275A704B7
:1033A700758307E559C4F582E0E0F573E0F574E04D
:1033B700F575E0F576E0F577E0F57875A700026238
:1033C7008CE59020E23EE5342437503812340C1255
:1033D70033E9205E4C7F2C90917012345090917796
:1033E7008067E534243775F009A42435FF205E068D
:1033F70024BE50027F3EEF249B50027F627E2674DC
:103407007112C769227D077F3312341E0F12341ED3
:10341700EF2408FFDDF3227E2F12D15BDEFB02D102
:103427005B7F2C120973E5BD123439E5BE123439BE
:10343700E5BFF8C412343FE8540775F007A490912C
:10344700622582F58250020583EF2409FF026BFA99
:1079F000027AA112D1E6E53724FC40F4B4FE14204B
:107A0000110EE590F45407600122E532247450EF22
:107A100002828A12D1E612C90E12C9A012C17D12C9
:107A2000C21D12C52A12C3737E197F3612C2C71235
:107A3000CE8F12C2DDC206E537600514602D804A84
:107A4000C23A127B45123C75123D3B1240B31249BB
:107A5000791249A1123927E54864186009E54824DC
:107A6000F6500312419E12D0FC8011D23A127B6B69
:107A700012345F123CE012BD3112D11412654F1264
:107A8000C9E71260AF126361800F127B5112BC7F95
:107A900012CABB12BD1512D0EC12822012C29F80F6
:107AA0000C12D1E6E53724F9401E127B2E30220954
:107AB0001233C8E5347002C222302309123BB9E503
:107AC000347002C22302D02612188F75170012CC10
:107AD000CE7F1212BDCB30124A75100075A7047507
:107AE0008306126347E51075F009A42415FFF51706
:107AF0007E00E512602F75F06484E5F00F12C6B9C0
:107B00001F7E0EE51112C1DB7516231264A105104C
:107B1000C3E55A95104006E51024F550BF30120316
:107B2000127BF18088745D12C76980D5C249302903
:107B300005121865800312188F909345127C04205B
:107B40002A71027BD7301223305E2030501D027E16
:107B5000E0301217305E06200B110284F712BDC40C
:027B60007F178D
:107B620012D00275172002CCCE12C88512C8263058
:107B7200120C20510302C8E512C10912BEE922E427
:107B8200FEFFE54824F6400D909768126C3F7E1682
:107B9200E54802C724B40E0690976E026C3F909798
:107BA20076126C3F7E12E54824F702C6BF7D208024
:107BB2000C7D3F302A077D633029027D3C7F0080A7
:107BC200247D2080127D3E800E7D3CE54975F007C4
:107BD200A42406800A7D3FE55975F007A42409FF15
:107BE20064027001FF7E1CED02C7377D2080027D9A
:107BF2003FE55B75F009A42416FF7E09ED02C73745
:107C0200C2497E207F00126C3F127B817E007F067C
:107C1200907D1F12C797E558B4FF012275100075B9
:107C2200A704758307126347E51075F007A42409BA
:107C3200FFF5177E00E51212C7377805EE2404FE21
:107C4200E012C737D8F67920E030E702792F3049C1
:107C520017120C8CFAB40408E510700C79658008D0
:107C6200EA14651070027923E97E1812C7377E2064
:107C7200E51230E70890936D126C3F8016E5111201
:107C82007CED1265012010052011028006301203DE
:107C9200127C9F0510C3E5589510508322127DA7D0
:087CA200127DBDFD7C00AE1C4B
:107CAA00AF1B125CF2BE003A8F00C3E57A9513FF50
:107CBA00E55E9514FE402B7C007D28125CFFC3EF25
:107CCA0098401F75F0058404FB24F950027B067E58
:107CDA002CAF170F12D12B0F12D12B0F12D12B0E43
:107CEA00DBEF2264B4602464B475F03284C0F0120D
:107CFA00C724CE2404CED0E075F00584C0F012C7A4
:107D0A0024CE2404CED0E02302C724907D1B026C2B
:107D1A003F2D2D2D000140FFFFFFE0FFFFFFFFC2B7
:107D2A005030123F20283CE558F4603720480320A1
:107D3A000931D250E559F51030330665586002050D
:107D4A0010127D71127DCD75A7049006DCE512F044
:107D5A00E511F0E517F0E510F075A7049006E0ECE0
:107D6A00F0EBF075A7002275A70475830712634725
:107D7A007813E0F608B819FA9006D07811E6F008F8
:107D8A00B819FAE51CF516F0E51BF515F0127DA7F2
:107D9A009006DAE514F0E513F075A7002275A7043A
